:020000040000FA
:06000000F4EF57F01200BE
:0A00060004008EB00000C1040000E9
:100010003A00000031B00000210F00000100000094
:1000200051B00000840400003D00000036B0000024
:08003000E10000001B000000CC
:08003800D9CFE6FFDACFE6FFA5
:10004000E1CFD9FFE2CFDAFFE652E652FC0EDBCF7A
:10005000DEFFDBCFDDFFF80EDBCF00F0DB06F90EB5
:10006000DBCF01F001E2DB06005001100CE0DFCF36
:10007000E9FFDF2A010EDBCFEAFF01E3DB2AFA0EFC
:10008000DBCFEFFFE8D7E552E552E552E5CFDAFFE7
:10009000E7CFD9FF1200D9CFE6FFDACFE6FFE1CFF5
:1000A000D9FFE2CFDAFF060EE12402E3E168E6526F
:1000B000E16EFC0EDBCFDEFFDBCFDDFFFA0EDBCF28
:1000C0003FF0FB0EDBCF40F0020E3FC0DBFF030E24
:1000D00040C0DBFF040EDB6A050EDB6AF80EDBCFE7
:1000E00000F0DB06F90EDBCF01F001E2DB06005089
:1000F000011022E0DFCFE9FFDF2A010EDBCFEAFFAC
:1001000001E3DB2AEFCF04F0020EDBCFE9FFDB2AAD
:10011000030EDBCFEAFF01E3DB2AEF50045C026E43
:10012000036A02BE0368040E02C0DBFF050E03C0B3
:10013000DBFF02500310D2E0040EDBCF00F0050E0F
:10014000DBCF01F000C0F3FF01C0F4FF060EE15C5D
:1001500002E2E16AE552E16EE552E5CFDAFFE7CF70
:10016000D9FF1200D9CFE6FFDACFE6FFE1CFD9FF02
:10017000E2CFDAFF0C0EE12402E3E168E652E16E21
:100180000A0EFEC4DBFF0B0EFFC4DBFFD950FA0FD3
:10019000E96EFF0EDA20EA6E020EEE5C000EEE58FB
:1001A000000EEE58000EEE5801E27FD2FA0EDBCFC1
:1001B00000F0FB0EDBCF01F0FC0EDBCF02F0FD0EFA
:1001C000DBCF03F00A0EDBCFE9FF0B0EDBCFEAFF3C
:1001D000060EE926000EEA22EE50005CEE500158B1
:1001E000EE500258EE50035801E35FD20A0EDBCF07
:1001F000E9FF0B0EDBCFEAFFEF50030A01E1ACD1C0
:10020000010A01E146D1030A01E04FD2FA0EDBCF29
:100210003FF0FB0EDBCF40F0020E3FC0DBFF030ED2
:1002200040C0DBFF020EDBCF00F0030EDBCF01F09E
:10023000010E0F0B05E0D89001320032E806FBE119
:10024000D950020FE96E000EDA20EA6E0050EE2659
:100250000150ED22020EDBCF00F0030EDBCF01F0E8
:100260000001010E0116040E00C0DBFF050E01C0E7
:10027000DBFFD950020FE96E000EDA20EA6E090E9C
:100280000F0B06E0EC52D890ED32EF32E806FAE1BF
:10029000D950040FE96E000EDA20EA6EFF0EEE1858
:1002A00002E1010EED183FE0020EE66EE66A040E72
:1002B000DBCFE6FF050EDBCFE6FF020EDBCF00F063
:1002C000030EDBCF01F0026A036A0A0EDBCFE9FFFF
:1002D0000B0EDBCFEAFF0A0EE926000EEA22EE50F3
:1002E0000026EE500122EE500222EE50032200C002
:1002F000E6FF01C0E6FF02C0E6FF03C0E6FFD950FB
:10030000060FE66E000EDA20E66E94EC4BF0046EFB
:100310000A0EE15C02E2E16AE552E16E0450000976
:1003200001E17FD0C2D1010EE66EE66AE668E66EB4
:10033000020EDBCF00F0030EDBCF01F0026A036A8E
:100340000A0EDBCFE9FF0B0EDBCFEAFF0A0EE92630
:10035000000EEA22EE500026EE500122EE5002225C
:10036000EE50032200C0E6FF01C0E6FF02C0E6FF38
:1003700003C0E6FFD950060FE66E000EDA20E66EE7
:1003800094EC4BF0046E0A0EE15C02E2E16AE55285
:10039000E16E0450000901E088D1010EE66EE66AC4
:1003A000000EE66EE66A020EDBCF04F0030EDBCF32
:1003B00005F0066A076A0A0EDBCFE9FF0B0EDBCFFA
:1003C000EAFF0A0EE926000EEA22EE500424006E2F
:1003D000EE500520016EEE500620026EEE50072012
:1003E000036E002A000E01220222032200C0E6FF53
:1003F00001C0E6FF02C0E6FF03C0E6FFD950070FC9
:10040000E66E000EDA20E66E94EC4BF0086E0A0EF3
:10041000E15C02E2E16AE552E16E0850000901E0A8
:1004200044D1070EDBCF02F002C003F0026A060ED1
:10043000DB500210DE6E03C0DDFF010E046E056AA4
:10044000066A076AD950FA0FE96EFF0EDA20EA6EE3
:10045000EE500416EE500516EE500616EE50071636
:1004600004500510061007100BE0DECF00F0DDCFC2
:1004700001F0040ED89001320032E804FBE169D0AB
:10048000DECF00F0DDCF01F0FF0E00160F0E0116DB
:1004900060D0020EE66EE66AFA0EDBCF00F0FB0ECD
:1004A0000001016A010ED89000360136E806FBE132
:1004B00000C0E6FF01C0E6FFFA0EDBCF02F0FB0E44
:1004C000DBCF03F0FC0EDBCF04F0FD0EDBCF05F03D
:1004D000080ED8900532043203320232E806F9E100
:1004E0000A0EDBCFE9FF0B0EDBCFEAFF0A0EE9268F
:1004F000000EEA22EE500226EE500322EE500422B5
:10050000EE50052202C0E6FF03C0E6FF04C0E6FF8E
:1005100005C0E6FFD950060FE66E000EDA20E66E43
:1005200094EC4BF0066E0A0EE15C02E2E16AE552E1
:10053000E16E0650000901E0B8D0070EDBCF04F0F1
:1005400004C005F0046A060EDB500410006E05C0FE
:1005500001F0026A036AA0D0040EE66EE66AFA0EA3
:10056000DBCF00F0FB0E0001016A009E020ED89066
:1005700000360136E806FBE100C0E6FF01C0E6FFF9
:10058000FA0EDBCF02F0FB0EDBCF03F0FC0EDBCF6D
:1005900004F0FD0EDBCF05F0070ED89005320432D3
:1005A00003320232E806F9E10A0EDBCFE9FF0B0E57
:1005B000DBCFEAFF0A0EE926000EEA22EE50022601
:1005C000EE500322EE500422EE50052202C0E6FF58
:1005D00003C0E6FF04C0E6FF05C0E6FFD950060FE2
:1005E000E66E000EDA20E66E94EC4BF0066E0A0E14
:1005F000E15C02E2E16AE552E16E0650000955E174
:10060000090EDBCF04F0056A066A076A180E1F0B95
:1006100007E0D8900436053606360736E806F9E1D5
:10062000080EDBCF08F0096A0A6A0B6A100E1F0B6E
:1006300007E0D890083609360A360B36E806F9E1A5
:1006400008500412095005120A5006120B500712E6
:10065000070EDBCF0CF00CC00DF00C6A0E6A0F6AAF
:100660000C5004120D5005120E5006120F500712B6
:10067000060EDBCF10F0116A126A136A04501010D4
:10068000006E05501110016E06501210026E0750D8
:100690001310036E0F0E031600C03DF001C03EF0B4
:1006A00002C03FF003C040F005D0010E3D6E3E6A2F
:1006B0003F6A406A0C0EE15C02E2E16AE552E16EDB
:1006C000E552E5CFDAFFE7CFD9FF1200D9CFE6FF39
:1006D000DACFE6FFE1CFD9FFE2CFDAFFE652E6520A
:1006E000FEC4DEFFFFC4DDFFD950FA0FE96EFF0E36
:1006F000DA20EA6E020EEE5E000EEE5AEE5AEE5A66
:10070000DECFE9FFDDCFEAFF060EE926000EEA2282
:10071000EECF00F0EECF01F0EECF02F0EFCF03F01E
:10072000020E005E000E015A025A035AD950FA0F07
:10073000E96EFF0EDA20EA6E0050EE5C0150EE58D2
:100740000250EE580350EE5805E33D6A3E6A3F6A98
:10075000406A46D0DECFE9FFDDCFEAFF120EE92680
:10076000000EEA22EECF08F0EECF09F0EECF0AF04D
:10077000EFCF0BF0DECFE9FFDDCFEAFF020EE92677
:10078000000EEA22EFCF04F0056A066A076A04C089
:100790003DF005C03EF006C03FF007C040F0FA0E45
:1007A000DBCF42F0FB0EDBCF43F0FC0EDBCF44F09F
:1007B000FD0EDBCF45F022EC57F039500824006ED7
:1007C0003A500920016E3B500A20026E3C500B202B
:1007D000036E00C03DF001C03EF002C03FF0406E2D
:1007E000E552E552E552E5CFDAFFE7CFD9FF120037
:1007F000D9CFE6FFDACFE6FFE1CFD9FFE2CFDAFFCC
:10080000060EE12402E3E168E652E16E040EFEC446
:10081000DBFF050EFFC4DBFFFC0EDBCFE9FFFD0EA7
:10082000DBCFEAFFEE6AED6AFC0EDBCFE9FFFD0EDF
:10083000DBCFEAFF040EE926000EEA22EECFDFFF4F
:10084000010EEECFDBFF020EEECFDBFF030EEECF8D
:10085000DBFFD9CFE9FFDACFEAFF010EEE1805E1A1
:10086000EE5003E1EE5001E1EE501FE0040EDBCF4D
:10087000E9FF050EDBCFEAFF060EE926000EEA22AD
:10088000EECF00F0EECF01F0EECF02F0EFCF03F0AD
:10089000D9CFE9FFDACFEAFF0050EE5C0150EE5805
:1008A0000250EE580350EE5802E3010E93D0D9CF18
:1008B000E9FFDACFEAFFEECF00F0EECF01F0EECFA6
:1008C00002F0EFCF03F000500110021003101EE100
:1008D000040EDBCFE9FF050EDBCFEAFFEF50030884
:1008E00015E1040EDBCFE9FF050EDBCFEAFF0E0EAC
:1008F000E926000EEA22EECFDFFF010EEECFDBFF8E
:10090000020EEECFDBFF030EEECFDBFFFC0EDBCFE4
:10091000E9FFFD0EDBCFEAFF080EE926000EEA2212
:10092000DFCFEEFF010EDBCFEEFF020EDBCFEEFFDF
:10093000030EDBCFEEFFD9CFE9FFDACFEAFFEECF30
:1009400004F0EECF05F0EECF06F0EFCF07F0045045
:100950000510061007101AE0D9CFE9FFDACFEAFF39
:10096000EECFE6FFEECFE6FFEECFE6FFEFCFE6FFFE
:10097000ADDEE552E552E552E5523DC000F03EC025
:1009800001F03FC002F040C003F012D0040EDBCFF4
:10099000E9FF050EDBCFEAFF0E0EE926000EEA2284
:1009A000EECF00F0EECF01F0EECF02F0EFCF03F08C
:1009B000FC0EDBCFE9FFFD0EDBCFEAFF0C0EE926D4
:1009C000000EEA2200C0EEFF01C0EEFF02C0EEFF03
:1009D00003C0EEFF006E060EE15C02E2E16AE55242
:1009E000E16E0050E552E5CFDAFFE7CFD9FF120004
:1009F000D9CFE6FFDACFE6FFE1CFD9FFE2CFDAFFCA
:100A0000080EE12402E3E168E652E16E060EFEC440
:100A1000DBFF070EFFC4DBFFFC0EDBCFE9FFFD0EA3
:100A2000DBCFEAFFEECF00F0EFCF01F0010E0026A2
:100A3000000E0122040E00C0DBFF050E01C0DBFF2B
:100A4000D950040FE96E000EDA20EA6EEE50ED1078
:100A500001E1D5D0FC0EDBCFE9FFFD0EDBCFEAFFD5
:100A60000C0EE926000EEA22EECF00F0EECF01F0E8
:100A7000EECF02F0EFCF03F0005001100210031090
:100A800001E1BDD0040EDBCF00F0050E016A0F0EB0
:100A900000160050011001E0F2D0FC0EDBCFE9FFA0
:100AA000FD0EDBCFEAFF0C0EE926000EEA22EE2A4D
:100AB000EE22EE22EE22FC0EDBCFE9FFFD0EDBCFB5
:100AC000EAFF080EE926000EEA22EECF00F0EECF94
:100AD00001F0EECF02F0EFCF03F000500110021052
:100AE00003101BE1040EDBCF00F0050EDBCF01F09D
:100AF000060EDBCFE9FF070EDBCFEAFF040EE92687
:100B0000000EEA22EECF02F0EFCF03F00250005CBD
:100B10000350015801E2B3D072D0040EDBCF02F0D3
:100B2000050EDBCF03F0040E0F0B05E0D890033267
:100B30000232E806FBE1060EDBCFE9FF070EDBCF52
:100B4000EAFF020EE926000EEA22EF040001021479
:100B5000006E016AE850011001E091D0FC0EDBCF7D
:100B6000E9FFFD0EDBCFEAFF080EE926000EEA22C0
:100B7000EECFE6FFEECFE6FFEECFE6FFEFCFE6FFEC
:100B8000B2EC00F0E552E552E552E5523DC0DEFF21
:100B90003EC0DEFF3FC0DEFF40C0DDFFDD52DD5264
:100BA000D9CFE9FFDACFEAFFD880010EEE54000E6C
:100BB000EE54000EEE54000EEE5402E3010E6CD023
:100BC000060EDBCFE9FF070EDBCFEAFF060EE926B4
:100BD000000EEA22EECF00F0EECF01F0EECF02F0F1
:100BE000EFCF03F0D9CFE9FFDACFEAFF0050EE5C98
:100BF0000150EE580250EE580350EE5802E3030E37
:100C00004BD0FC0EDBCFE9FFFD0EDBCFEAFF080E79
:100C1000E926000EEA22DFCFEEFF010EDBCFEEFF6A
:100C2000020EDBCFEEFF030EDBCFEEFFD9CFE9FFE5
:100C3000DACFEAFFEECFE6FFEECFE6FFEECFE6FF3C
:100C4000EFCFE6FF43DDE552E552E552E5523EC007
:100C500001F03FC002F040C003F0FC0EDBCFE9FF23
:100C6000FD0EDBCFEAFF0C0EE926000EEA223DC0A6
:100C7000EEFF01C0EEFF02C0EEFF03C0EEFFFC0E70
:100C8000DBCFE9FFFD0EDBCFEAFF040EDBCFEEFF8B
:100C9000050EDBCFEDFF000E006E080EE15C02E2F8
:100CA000E16AE552E16E0050E552E5CFDAFFE7CFA9
:100CB000D9FF1200D9CFE6FFDACFE6FFE1CFD9FFA7
:100CC000E2CFDAFFE652E652FC0EDBCFE6FFFD0E86
:100CD000DBCFE6FF8DDDE552E552DF6EDF5002E04F
:100CE000DF5098D0200EE66EE66AFC0EDBCFE9FFFF
:100CF000FD0EDBCFEAFFEECF00F0EFCF01F00001F9
:100D0000016A0F0E0016050ED89000360136E8066F
:100D1000FBE100C0E6FF01C0E6FFFC0EDBCFE9FF10
:100D2000FD0EDBCFEAFF0C0EE926000EEA22EECF25
:100D3000E6FFEECFE6FFEECFE6FFEFCFE6FFFA0EDF
:100D4000DBCFE6FFFB0EDBCFE6FF94EC4BF0026E51
:100D50000A0EE15C02E2E16AE552E16E025000092E
:100D600002E0010E01D0000EDF6EDF5052E1FA0EFC
:100D7000DBCFE9FFFB0EDBCFEAFF010EEFCFDBFF9E
:100D8000DB5003E1030EDF6E44D00B0EE76EFA0E6C
:100D9000DBCFE9FFFB0EDBCFEAFFE750E926000ED1
:100DA000EA22EF50080B28E10B0EE66EE66AFC0E15
:100DB000DBCFE9FFFD0EDBCFEAFF020EE926000ED6
:100DC000EA22EECFE6FFEFCFE6FFFA0EDBCFE6FF3B
:100DD000FB0EDBCFE6FF4BEC00F0026E060EE15C93
:100DE00002E2E16AE552E16E0250F3CF00F0F4CF87
:100DF00001F0F350F4100DE0FC0EDBCFE6FFFD0E2A
:100E0000DBCFE6FFF5DDE552E552DF6EDF5001E1B5
:100E100069D7DF50E552E552E552E5CFDAFFE7CF7B
:100E2000D9FF1200D9CFE6FFDACFE6FFE1CFD9FF35
:100E3000E2CFDAFF090EE12402E3E168E652E16E57
:100E4000FC0EDBCFE9FFFD0EDBCFEAFF020EE92649
:100E5000000EEA22050EEECFDBFF060EEDCFDBFF24
:100E60000B0EE66EE66A200EE66EE66A050EDBCF36
:100E7000E6FF060EDBCFE6FF1CEC00F0006E060E70
:100E8000E15C02E2E16AE552E16E0050040EDB6AC9
:100E9000030EDB6A080EF36E020EF3CFDBFFFA0ED1
:100EA000DBCFE9FFFB0EDBCFEAFF070EEECFDBFF68
:100EB000080EEDCFDBFF030EDBCFF3FFDB2AF35091
:100EC000E76E070EDBCFE9FF080EDBCFEAFFE75046
:100ED000E926000EEA22EFCFDFFFDF5020083CE2D8
:100EE0002F0EDF5C39E02E0EDF5C09E0020EDB50D6
:100EF000F36E040EDBCFF4FFF350F45C12E3020E4A
:100F0000DB50080829E12E0EDF5C26E1080EF36EA7
:100F1000040EF3CFDBFF0B0EF36E020EF3CFDBFFFD
:100F2000CAD7610EDF5C05E3DF507A0802E3200ECA
:100F3000DF5E040EDBCFF3FFDB2AF350E76E050E16
:100F4000DBCFE9FF060EDBCFEAFFE750E926000E14
:100F5000EA22DFCFEFFFAFD7030EDB50E76E070EBD
:100F6000DBCF00F0080EDBCF01F0E7500026000ECB
:100F70000122FA0EDBCFE9FFFB0EDBCFEAFF00C058
:100F8000EEFF01C0EDFFDF50200802E3010E01D0AB
:100F9000000EE66E0B0EE76E050EDBCFE9FF060EC8
:100FA000DBCFEAFFE750E926000EEA22E552E750E0
:100FB000EF6E000E006E090EE15C02E2E16AE5529E
:100FC000E16E0050E552E5CFDAFFE7CFD9FF12001E
:100FD000D9CFE6FFDACFE6FFE1CFD9FFE2CFDAFFE4
:100FE000E652F80EDBCFE9FFF90EDBCFEAFFEF5058
:100FF000200806E1F80EDB2AF90EF3E3DB2AF1D72D
:10100000F80EDBCFE9FFF90EDBCFEAFFEF502F0838
:1010100005E1F80EDB2AF90E01E3DB2AFC0EDBCF3B
:10102000E9FFFD0EDBCFEAFF040EE926000EEA22FF
:10103000EE6AEE6AEE6AEE6AF80EDBCFE9FFF90EB1
:10104000DBCFEAFFEF50200813E3FC0EDBCFE6FF17
:10105000FD0EDBCFE6FFF8EC03F0E552E552DF6E64
:10106000FA0EDBCFE9FFFB0EDBCFEAFFEF6AE0D041
:10107000D950F80FE66EFF0EDA20E66EFC0EDBCFDD
:10108000E6FFFD0EDBCFE6FFCDDEE552E552E55291
:10109000E552DF6EDF5001E0CBD0FA0EDBCFE6FF8A
:1010A000FB0EDBCFE6FFFC0EDBCFE6FFFD0EDBCF5A
:1010B000E6FF00DEE552E552E552E552DF6EDF5015
:1010C0001AE0030EDF5C01E0B3D0FC0EDBCFE9FFDA
:1010D000FD0EDBCFEAFF020EE926000EEA22EE50FB
:1010E000EFCFEAFFE96E0B0EE926000EEA22EF5081
:1010F00001E09ED024D0FC0EDBCFE9FFFD0EDBCF5C
:10110000EAFF020EE926000EEA22EE50EFCFEAFFD8
:10111000E96E0B0EE926000EEA22EF5001E088D0BE
:101120000B0EE76EFA0EDBCFE9FFFB0EDBCFEAFF1B
:10113000E750E926000EEA22EF50100B03E1040EFF
:10114000DF6E76D0140EE76EFA0EDBCFE9FFFB0EF2
:10115000DBCFEAFFE750E926000EEA22010EE9267E
:10116000000EEA22EFCF04F004C005F0046A140E6A
:10117000E76EFA0EDBCFE9FFFB0EDBCFEAFFE750AD
:10118000E926000EEA22EF500410006E05C001F0BF
:10119000026A036A100E1F0B07E0D8900036013672
:1011A00002360336E806F9E11A0EE76EFA0EDBCFD7
:1011B000E9FFFB0EDBCFEAFFE750E926000EEA224B
:1011C000010EE926000EEA22EFCF0AF00AC00BF06A
:1011D0000A6A1A0EE76EFA0EDBCFE9FFFB0EDBCFD1
:1011E000EAFFE750E926000EEA22EF5000010A105C
:1011F000066E0BC007F0086A096AE85000120B502F
:1012000001120850021209500312FC0EDBCFE9FF55
:10121000FD0EDBCFEAFF040EE926000EEA2200C035
:10122000EEFF01C0EEFF02C0EEFF03C0EEFF20D7CD
:10123000DF50E552E552E5CFDAFFE7CFD9FF1200E4
:10124000D9CFE6FFDACFE6FFE1CFD9FFE2CFDAFF71
:10125000020EE66EE66AFE0EE66E010EE66ED950EE
:10126000F80FE96EFF0EDA20EA6EEECFE6FFEECF62
:10127000E6FFEECFE6FFEFCFE6FFFC0EDBCFE6FFAB
:10128000FD0EDBCFE6FF94EC4BF0006E0A0EE15C46
:1012900002E2E16AE552E16E0050000902E0030E4D
:1012A000BAD0010EE76EFC0EDBCFE9FFFD0EDBCFFF
:1012B000EAFFE750E926000EEA22EFCF02F002C073
:1012C00003F0026AFC0EDBCFE9FFFD0EDBCFEAFF85
:1012D000EF5000010210006E03C001F0550E00181F
:1012E00002E1AA0E011802E0020E95D0020EE66E8F
:1012F000E66A360EE66EE66AD950F80FE96EFF0E22
:10130000DA20EA6EEECFE6FFEECFE6FFEECFE6FFA5
:10131000EFCFE6FFFC0EDBCFE6FFFD0EDBCFE6FFF7
:1013200094EC4BF0006E0A0EE15C02E2E16AE552D9
:10133000E16E0050000923E1010EE76EFC0EDBCFE9
:10134000E9FFFD0EDBCFEAFFE750E926000EEA22B7
:10135000EFCF03F003C004F0036AFC0EDBCFE9FF1C
:10136000FD0EDBCFEAFFEF5000010310016E04C059
:1013700002F0460E011803E1410E021849E0020E88
:10138000E66EE66A520EE66EE66AD950F80FE96E2E
:10139000FF0EDA20EA6EEECFE6FFEECFE6FFEECFED
:1013A000E6FFEFCFE6FFFC0EDBCFE6FFFD0EDBCF67
:1013B000E6FF94EC4BF0006E0A0EE15C02E2E16A9B
:1013C000E552E16E0050000925E1010EE76EFC0ECA
:1013D000DBCFE9FFFD0EDBCFEAFFE750E926000E89
:1013E000EA22EFCF03F003C004F0036AFC0EDBCF68
:1013F000E9FFFD0EDBCFEAFFEF5000010310016EA5
:1014000004C002F0460E011805E1410E021802E187
:10141000000E01D0010EE552E5CFDAFFE7CFD9FF8C
:101420001200D9CFE6FFDACFE6FFE1CFD9FFE2CF56
:10143000DAFF350EE12402E3E168E652E16E0401D1
:10144000FE6BFF6BD950FC0FE96EFF0EDA20EA6EDF
:10145000EE50ED1002E10EEF0FF029EC4AF0010B17
:1014600003E0020E0FEF0FF0250EDB6A260EDB6A9B
:10147000270EDB6A280EDB6AD950250FE96E000EB5
:10148000DA20EA6EEECFE6FFEECFE6FFEECFE6FF24
:10149000EFCFE6FFD950010FE66E000EDA20E66EC0
:1014A000CFDE006E060EE15C02E2E16AE552E16E1B
:1014B0000050DF6EDF0401E09CD0100EE66EE66A9D
:1014C000BE0EE66E010EE66ED950250FE96E000ED7
:1014D000DA20EA6EEECFE6FFEECFE6FFEECFE6FFD4
:1014E000EFCFE6FFD950010FE66E000EDA20E66E70
:1014F00094EC4BF0006E0A0EE15C02E2E16AE55208
:10150000E16E0050000902E0030E72D0050EDB50C0
:1015100070E00C0EDBCF00F0016A026A036A180E5D
:101520001F0B07E0D8900036013602360336E80676
:10153000F9E10B0EDBCF04F0056A066A076A100EAC
:101540001F0B07E0D8900436053606360736E80646
:10155000F9E1045000120550011206500212075022
:1015600003120A0EDBCF08F008C009F0086A0A6A05
:101570000B6A08500012095001120A5002120B5057
:101580000312090EDBCF0CF00D6A0E6A0F6A0C50C5
:1015900000120D5001120E5002120F500312250EB0
:1015A00000C0DBFF260E01C0DBFF270E02C0DBFF01
:1015B000280E03C0DBFFD950250FE96E000EDA209C
:1015C000EA6EEECFE6FFEECFE6FFEECFE6FFEFCF1F
:1015D000E6FFD950010FE66E000EDA20E66E30DE2F
:1015E000006E060EE15C02E2E16AE552E16E005037
:1015F000DF6E030EDF5C2BE0DF5003E0070E0FEF22
:101600000FF0240EE66EE66A0D0EE66EE66AD9501D
:10161000250FE96E000EDA20EA6EEECFE6FFEECF80
:10162000E6FFEECFE6FFEFCFE6FFD950010FE66E03
:10163000000EDA20E66E94EC4BF0006E0A0EE15CD0
:1016400002E2E16AE552E16E0050000902E0010E9B
:10165000E6D3D950170FE96E000EDA20EA6E0D0EB0
:10166000E95E000EEA5A010EE926000EEA22EFCFEB
:1016700002F002C003F0026AD950170FE96E000EA3
:10168000DA20EA6E0D0EE95E000EEA5AEF50000114
:101690000210006E290E00C0DBFF2A0E03C0DBFF24
:1016A0002B0EDB6A2C0EDB6A290EDBCF00F02A0E34
:1016B000DBCF01F02B0EDBCF02F02C0EDBCF03F0E3
:1016C000005001100210031001E082D0D950250F04
:1016D000E96E000EDA20EA6E0D0EE95E000EEA5A9F
:1016E000030EE926000EEA22EFCF00F0016A026A3B
:1016F000036A180E1F0B07E0D89000360136023639
:101700000336E806F9E1D950250FE96E000EDA201C
:10171000EA6E0D0EE95E000EEA5A020EE926000E90
:10172000EA22EFCF04F0056A066A076A100E1F0B63
:1017300007E0D8900436053606360736E806F9E1A4
:1017400004500012055001120650021207500312F5
:10175000D950250FE96E000EDA20EA6E0D0EE95E13
:10176000000EEA5A010EE926000EEA22EFCF08F039
:1017700008C009F0086A0A6A0B6A0850001209508A
:1017800001120A5002120B500312D950250FE96EB4
:10179000000EDA20EA6E0D0EE95E000EEA5AEFCF77
:1017A0000CF00D6A0E6A0F6A0C5000120D500112F7
:1017B0000E5002120F500312290E00C0DBFF2A0E3A
:1017C00001C0DBFF2B0E02C0DBFF2C0E03C0DBFFD2
:1017D000040EDBCF00F0016A026A036AD950290FB8
:1017E000E96E000EDA20EA6E00C042F001C043F05C
:1017F00002C044F003C045F0EECF3DF0EECF3EF026
:10180000EECF3FF0EFCF40F022EC57F03CC0EDFFC1
:101810003BC0EDFF3AC0EDFF39C0EFFFD9500F0FCD
:10182000E96E000EDA20EA6E0D0EE95E000EEA5A4D
:10183000010EE926000EEA22EFCF04F004C005F005
:10184000046AD9500F0FE96E000EDA20EA6E0D0E11
:10185000E95E000EEA5AEF500410006E05C001F078
:10186000026A036AD950250FE96E000EDA20EA6E8B
:10187000EE500026EE500122EE500222EE500322DE
:10188000FC0EDBCFE9FFFD0EDBCFEAFF0A0EE926F7
:10189000000EEA2200C0EEFF01C0EEFF02C0EEFF24
:1018A00003C0EEFFFC0EDBCFE9FFFD0EDBCFEAFF4E
:1018B000020EE926000EEA22010EDBCFEFFFD9501F
:1018C000120FE96E000EDA20EA6E0D0EE95E000ED0
:1018D000EA5A010EE926000EEA22EFCF02F002C01A
:1018E00003F0026AD950120FE96E000EDA20EA6E98
:1018F0000D0EE95E000EEA5AEF500210006E03C0B2
:1019000001F0FC0EDBCFE9FFFD0EDBCFEAFF040E9A
:10191000E926000EEA2200C0EEFF01C0EDFFD9501B
:10192000140FE96E000EDA20EA6E0D0EE95E000E6D
:10193000EA5A010EE926000EEA22EFCF02F002C0B9
:1019400003F0026AD950140FE96E000EDA20EA6E35
:101950000D0EE95E000EEA5AEF500210006E2D0ED9
:1019600000C0DBFF2E0E03C0DBFF2F0EDB6A300E44
:10197000DB6A2D0EDBCF00F02E0EDBCF01F02F0E39
:10198000DBCF02F0300EDBCF03F00050011002106D
:10199000031001E082D0D950210FE96E000EDA2049
:1019A000EA6E0D0EE95E000EEA5A030EE926000EFD
:1019B000EA22EFCF00F0016A026A036A180E1F0BD9
:1019C00007E0D8900036013602360336E806F9E122
:1019D000D950210FE96E000EDA20EA6E0D0EE95E95
:1019E000000EEA5A020EE926000EEA22EFCF04F0BA
:1019F000056A066A076A100E1F0B07E0D8900436C6
:101A0000053606360736E806F9E10450001205509F
:101A100001120650021207500312D950210FE96E2D
:101A2000000EDA20EA6E0D0EE95E000EEA5A010E93
:101A3000E926000EEA22EFCF08F008C009F0086A94
:101A40000A6A0B6A08500012095001120A50021269
:101A50000B500312D950210FE96E000EDA20EA6E06
:101A60000D0EE95E000EEA5AEFCF0CF00D6A0E6A19
:101A70000F6A0C5000120D5001120E5002120F503E
:101A800003122D0E00C0DBFF2E0E01C0DBFF2F0E58
:101A900002C0DBFF300E03C0DBFFFC0EDBCFE9FF33
:101AA000FD0EDBCFEAFF020EE926000EEA22EFCFA1
:101AB0001AF01B6A1C6A1D6AD9500F0FE96E000EDE
:101AC000DA20EA6E0D0EE95E000EEA5A010EE926F2
:101AD000000EEA22EFCF14F014C015F0146AD950AA
:101AE0000F0FE96E000EDA20EA6E0D0EE95E000EB1
:101AF000EA5AEF5000011410106E15C011F0126A6E
:101B0000136AD9502D0FE96E000EDA20EA6E1050DC
:101B1000EE5C0C6E1550EE580D6E1250EE580E6EB7
:101B20001350EE580F6ED950290FE96E000EDA20CF
:101B3000EA6EEE500C5C086EEE500D58096EEE50D9
:101B40000E580A6EEE500F580B6EFC0EDBCFE9FFFD
:101B5000FD0EDBCFEAFF040EE926000EEA22EECFEF
:101B600016F0EFCF17F0040E0F0B05E0D8901732E8
:101B70001632E806FBE1186A196A1650085C046E12
:101B800017500958056E18500A58066E19500B5810
:101B9000076E04C03DF005C03EF006C03FF0406E49
:101BA0001AC042F01BC043F01CC044F01DC045F0F9
:101BB00087EC57F03DC000F03EC001F03FC002F09E
:101BC00040C003F0020E0026000E01220222032272
:101BD000310E00C0DBFF320E01C0DBFF330E02C04E
:101BE000DBFF340E03C0DBFFFC0EDBCFE9FFFD0E95
:101BF000DBCFEAFF060EE926000EEA22310EDBCF2C
:101C0000EEFF320EDBCFEEFF330EDBCFEEFF340EF6
:101C1000DBCFEEFF020EDF6ED950310FE96E000E02
:101C2000DA20EA6EF70EEE5C0F0EEE58000EEE585C
:101C3000000EEE5802E2010EDF6ED950310FE96E50
:101C4000000EDA20EA6EF70EEE5CFF0EEE58000E84
:101C5000EE58000EEE5802E3030EDF6EFC0EDBCFF3
:101C6000E9FFFD0EDBCFEAFFDFCFEFFF030EDF5C06
:101C700047E1230EDBCF00F0016A026A036A180E07
:101C80001F0B07E0D8900036013602360336E8060F
:101C9000F9E1220EDBCF04F0056A066A076A100E2E
:101CA0001F0B07E0D8900436053606360736E806DF
:101CB000F9E10450001205500112065002120750BB
:101CC0000312210EDBCF08F008C009F0086A0A6A87
:101CD0000B6A08500012095001120A5002120B50F0
:101CE0000312200EDBCF0CF00D6A0E6A0F6A0C5047
:101CF00000120D5001120E5002120F5003121ED08E
:101D0000290EDBCF00F02A0EDBCF01F02B0EDBCF4C
:101D100002F02C0EDBCF03F0FC0EDBCFE9FFFD0E53
:101D2000DBCFEAFF0A0EE926000EEA22EE5000267B
:101D3000EE500122EE500222EE500322FC0EDBCFC9
:101D4000E9FFFD0EDBCFEAFF0E0EE926000EEA22C8
:101D500000C0EEFF01C0EEFF02C0EEFF03C0EEFFC9
:101D6000290EDBCF00F02A0EDBCF01F02B0EDBCFEC
:101D700002F02C0EDBCF03F0FC0EDBCFE9FFFD0EF3
:101D8000DBCFEAFF0A0EE926000EEA22EE5000261B
:101D9000EE500122EE500222EE500322FC0EDBCF69
:101DA000E9FFFD0EDBCFEAFF040EE926000EEA2272
:101DB000EECF04F0EFCF05F0040E0F0B05E0D89046
:101DC00005320432E806FBE1066A076A0450002681
:101DD000055001220650022207500322FC0EDBCFE1
:101DE000E9FFFD0EDBCFEAFF120EE926000EEA2224
:101DF00000C0EEFF01C0EEFF02C0EEFF03C0EEFF29
:101E0000FC0EDBCFE9FFFD0EDBCFEAFFEE52EF6AFF
:101E1000FC0EDBCFFEF4FD0EDBCFFFF4000E006EF8
:101E2000350EE15C02E2E16AE552E16E0050E552F6
:101E3000E5CFDAFFE7CFD9FF1200D9CFE6FFDACF3F
:101E4000E6FFE1CFD9FFE2CFDAFF3F0EE12402E364
:101E5000E168E652E16E3D0EFEC4DBFF3E0EFFC4BC
:101E6000DBFFD9503D0FE96E000EDA20EA6EEE502E
:101E7000ED1002E1060EEBD03D0EDBCFE9FF3E0E8A
:101E8000DBCFEAFFEE52EF6AD950110F006E000E61
:101E9000DA20016E030E00C0DBFF040E01C0DBFF81
:101EA000FC0EDBCFE6FFFD0EDBCFE6FFD9501D0FAA
:101EB000E66E000EDA20E66ED950010FE66E000ED7
:101EC000DA20E66EE8EC07F0006E060EE15C02E256
:101ED000E16AE552E16E0050DF6EDF5002E0DF5054
:101EE000B6D01D0EDB5004E0280EDB50100B02E0D4
:101EF000030EADD0320EDBCF04F004C005F0046A4F
:101F0000310EDB500410006E05C001F0026A036A56
:101F1000100E1F0B07E0D89000360136023603364C
:101F2000E806F9E1380EDBCF0AF00AC00BF00A6AC6
:101F3000370EDB500A10086A096AE85000120B508D
:101F4000011208500212095003123D0EDBCFE9FFC7
:101F50003E0EDBCFEAFF1E0EE926000EEA2200C08D
:101F6000EEFF01C0EEFF02C0EEFF03C0EEFF3C0E2D
:101F7000DBCF00F0016A026A036A180E1F0B07E04C
:101F8000D8900036013602360336E806F9E13B0EFA
:101F9000DBCF04F0056A066A076A100E1F0B07E024
:101FA000D8900436053606360736E806F9E10450BF
:101FB00000120550011206500212075003123A0E89
:101FC000DBCF08F008C009F0086A0A6A0B6A0850FB
:101FD0000012095001120A5002120B500312390E5E
:101FE000DBCF0CF00D6A0E6A0F6A0C5000120D5018
:101FF00001120E5002120F5003123D0EDBCFE9FF0B
:102000003E0EDBCFEAFF1A0EE926000EEA2200C0E0
:10201000EEFF01C0EEFF02C0EEFF03C0EEFF3D0E7B
:10202000DBCFE9FF3E0EDBCFEAFF160EE926000EFE
:10203000EA22EE6AEE6AEE6AEE6A3D0EDBCFE9FF57
:102040003E0EDBCFEAFFEE52010EEF6E000E006E89
:102050003F0EE15C02E2E16AE552E16E0050E552BA
:10206000E5CFDAFFE7CFD9FF1200D9CFE6FFDACF0D
:10207000E6FFE1CFD9FFE2CFDAFF140EE12402E35D
:10208000E168E652E16EFC0EDBCF3FF0FD0EDBCFE8
:1020900040F0100E3FC0DBFF110E40C0DBFF120E00
:1020A000FEC4DBFF130EFFC4DBFFF80EDBCFE9FF3E
:1020B000F90EDBCFEAFFEE6AED6AD950120FE96E36
:1020C000000EDA20EA6EEE50ED1002E1060E87D225
:1020D000120EDBCFE9FF130EDBCFEAFFEE52EF501B
:1020E000010B02E1050E7BD2120EDBCFE9FF130ECE
:1020F000DBCFEAFF1A0EE926000EEA22EECF04F04B
:10210000EECF05F0EECF06F0EFCF07F0120EDBCFEB
:10211000E9FF130EDBCFEAFF160EE926000EEA22D6
:10212000EE50045C006EEE500558016EEE500658FD
:10213000026EEE500758036E090E00C0DBFF0A0E58
:1021400001C0DBFF0B0E02C0DBFF0C0E03C0DBFF88
:10215000FA0EDBCF00F0FB0EDBCF01F0026A036A60
:10216000D950090FE96E000EDA20EA6E0050EE5CDD
:102170000150EE580250EE580350EE580CE2090E92
:10218000DBCF3FF00A0EDBCF40F0FA0E3FC0DBFFA3
:10219000FB0E40C0DBFFD950FA0FE96EFF0EDA20CC
:1021A000EA6EEE50ED1001E10FD2120EDBCFE9FF27
:1021B000130EDBCFEAFF160EE926000EEA22EECF61
:1021C00000F0EECF01F0010E0116026A036A005022
:1021D00001100210031001E010D1120EDBCFE9FF55
:1021E000130EDBCFEAFF160EE926000EEA22EECF31
:1021F00000F0EECF01F0EECF02F0EFCF03F0090ECA
:10220000D8900332023201320032E806F9E1120EB0
:10221000DBCFE9FF130EDBCFEAFF020EE926000E4B
:10222000EA22EF04046E056A066A076AE85000169F
:102230000550011606500216075003160F0E00C077
:10224000DBFFDB5001E07DD0120EDBCFE9FF130E88
:10225000DBCFEAFF160EE926000EEA22EECF04F0ED
:10226000EECF05F0EECF06F0EFCF07F004500510EB
:102270000610071013E1120EDBCFE9FF130EDBCFC0
:10228000EAFF1E0EE926000EEA22EECF00F0EECFA6
:1022900001F0EECF02F0EFCF03F020D0120EDBCF33
:1022A000E9FF130EDBCFEAFF220EE926000EEA2239
:1022B000EECFE6FFEECFE6FFEECFE6FFEFCFE6FF95
:1022C000B2EC00F0E552E552E552E5523DC000F0B7
:1022D0003EC001F03FC002F040C003F0010E00C05C
:1022E000DBFF020E01C0DBFF030E02C0DBFF040EAA
:1022F00003C0DBFFD950010FE96E000EDA20EA6E51
:10230000D880010EEE54000EEE54000EEE54000E76
:10231000EE5401E35BD1120EDBCFE9FF130EDBCFEE
:10232000EAFF220EE926000EEA22010EDBCFEEFFC5
:10233000020EDBCFEEFF030EDBCFEEFF040EDBCF92
:10234000EEFF120EDBCFE9FF130EDBCFEAFF220E0A
:10235000E926000EEA22EECFE6FFEECFE6FFEECF53
:10236000E6FFEFCFE6FF66EC03F0E552E552E552FB
:10237000E552050E3DC0DBFF060E3EC0DBFF070E3B
:102380003FC0DBFF080E40C0DBFF050EDBCF00F0D7
:10239000060EDBCF01F0070EDBCF02F0080EDBCF1D
:1023A00003F0005001100210031001E10FD10F0ED5
:1023B000DBCF00F0016A026A036AD950050FE96EAB
:1023C000000EDA20EA6EEE500026EE500122EE50AA
:1023D0000222EE500322120EDBCFE9FF130EDBCFF9
:1023E000EAFF260EE926000EEA2200C0EEFF01C039
:1023F000EEFF02C0EEFF03C0EEFF046A020E056EA0
:10240000066A076A120EDBCFE9FF130EDBCFEAFF85
:10241000160EE926000EEA22EECF3DF0EECF3EF09A
:10242000EECF3FF0EFCF40F0426A020E436E446AB7
:10243000456A87EC57F03950045C006E3A500558F5
:10244000016E3B5006583C5007580D0E00C0DBFF94
:102450000E0E01C0DBFF0D0EDBCF00F00E0EDBCF4A
:1024600001F0FA0EDBCF02F0FB0EDBCF03F00050E1
:10247000025C015003580CE2FA0EDBCF3FF0FB0E7A
:10248000DBCF40F00D0E3FC0DBFF0E0E40C0DBFF88
:102490000D0EDBCFE6FF0E0EDBCFE6FF120EDBCF1D
:1024A000E9FF130EDBCFEAFF160EE926000EEA2243
:1024B000EECF00F0EECF01F0010E0116026A036AC2
:1024C00000C0E6FF01C0E6FF120EDBCFE9FF130EEE
:1024D000DBCFEAFF260EE926000EEA22EECFE6FF6A
:1024E000EECFE6FFEECFE6FFEFCFE6FFD950FC0FD1
:1024F000E96EFF0EDA20EA6EEE50ED1003E1046A99
:10250000056A06D0100EDBCF04F0110EDBCF05F00C
:1025100004C0E6FF05C0E6FF94EC4BF0066E0A0E21
:10252000E15C02E2E16AE552E16E0650DF6EDF50E7
:102530004DE10D0EDBCF00F00E0EDBCF01F0026A95
:10254000036A120EDBCFE9FF130EDBCFEAFF160E94
:10255000E926000EEA220050EE260150EE2202503B
:10256000EE220350EE220D0EDBCF00F00E0EDBCF7D
:1025700001F0D950100FE96E000EDA20EA6E00501B
:10258000EE260150ED220D0EDBCF00F00E0EDBCF5C
:1025900001F0D950FA0FE96EFF0EDA20EA6E005012
:1025A000EE5E0150ED5A0D0EDBCF00F00E0EDBCFCC
:1025B00001F0F80EDBCFE9FFF90EDBCFEAFF0050A8
:1025C000EE260150ED22E7D5000E09D0120EDBCF2A
:1025D000E9FF130EDBCFEAFFEE52EF6A010E006E49
:1025E000140EE15C02E2E16AE552E16E0050E55250
:1025F000E5CFDAFFE7CFD9FF1200D9CFE6FFDACF78
:10260000E6FFE1CFD9FFE2CFDAFF130EE12402E3C8
:10261000E168E652E16EFC0EDBCF3FF0FD0EDBCF52
:1026200040F00C0E3FC0DBFF0D0E40C0DBFF110E73
:10263000FEC4DBFF120EFFC4DBFFF80EDBCFE9FFA9
:10264000F90EDBCFEAFFEE6AED6AD950110FE96EA1
:10265000000EDA20EA6EEE50ED1002E1060EDFD237
:10266000110EDBCFE9FF120EDBCFEAFFEE52EF5087
:10267000010B02E1050ED3D2D950FA0FE96EFF0E1D
:10268000DA20EA6EEE50ED1027E1110EDBCFE9FF04
:10269000120EDBCFEAFFEE52EF50400B14E0E66A79
:1026A000E66AE66AE66A000EE66EE66A65EC4CF0FB
:1026B000006E060EE15C02E2E16AE552E16E005056
:1026C000000901E0A3D2110EDBCFE9FF120EDBCF30
:1026D000EAFFEE52EF9C98D2110EDBCFE9FF120E0B
:1026E000DBCFEAFFEE52EF50400B0CE1110EDBCFD7
:1026F000E9FF120EDBCFEAFF160EE926000EEA22F2
:10270000EE6AEE90110EDBCFE9FF120EDBCFEAFF8F
:102710001A0EE926000EEA22EECF04F0EECF05F005
:10272000EECF06F0EFCF07F0110EDBCFE9FF120E70
:10273000DBCFEAFF160EE926000EEA22EE50045C1B
:10274000006EEE500558016EEE500658026EEE50C7
:102750000758036E080E00C0DBFF090E01C0DBFF47
:102760000A0E02C0DBFF0B0E03C0DBFFFA0EDBCF4D
:1027700000F0FB0EDBCF01F0026A036AD950080FAC
:10278000E96E000EDA20EA6E0050EE5C0150EE5861
:102790000250EE580350EE580CE2080EDBCF3FF02B
:1027A000090EDBCF40F0FA0E3FC0DBFFFB0E40C04E
:1027B000DBFFD950FA0FE96EFF0EDA20EA6EEE5019
:1027C000ED1001E121D2110EDBCFE9FF120EDBCFBC
:1027D000EAFF160EE926000EEA22EECF00F0EFCF58
:1027E00001F00001010E01160050011001E035D189
:1027F000110EDBCFE9FF120EDBCFEAFF160EE92642
:10280000000EEA22EECF00F0EECF01F0EECF02F0A4
:10281000EFCF03F0090ED8900332023201320032BA
:10282000E806F9E1110EDBCFE9FF120EDBCFEAFF7C
:10283000020EE926000EEA22EF04046E056A066A1B
:10284000076AE85000160550011606500216075098
:1028500003160E0E00C0DBFFDB5001E079D0110E35
:10286000DBCFE9FF120EDBCFEAFF160EE926000EE2
:10287000EA22EECF04F0EECF05F0EECF06F0EFCF78
:1028800007F0045005100610071013E1110EDBCFFE
:10289000E9FF120EDBCFEAFF1E0EE926000EEA2248
:1028A000EECF00F0EECF01F0EECF02F0EFCF03F06D
:1028B00020D0110EDBCFE9FF120EDBCFEAFF220E94
:1028C000E926000EEA22EECFE6FFEECFE6FFEECFDE
:1028D000E6FFEFCFE6FFB2EC00F0E552E552E5523D
:1028E000E5523DC000F03EC001F03FC002F040C0E4
:1028F00003F000C0DFFF010E01C0DBFF020E02C0CB
:10290000DBFF030E03C0DBFFD9CFE9FFDACFEAFF1D
:10291000D880010EEE54000EEE54000EEE54000E60
:10292000EE5401E373D1110EDBCFE9FF120EDBCFC2
:10293000EAFF220EE926000EEA22DFCFEEFF010EAB
:10294000DBCFEEFF020EDBCFEEFF030EDBCFEEFFA1
:10295000110EDBCFE9FF120EDBCFEAFF220EE926D4
:10296000000EEA22EECFE6FFEECFE6FFEECFE6FF67
:10297000EFCFE6FF66EC03F0E552E552E552E55293
:10298000040E3DC0DBFF050E3EC0DBFF060E3FC060
:10299000DBFF070E40C0DBFF040EDBCF00F0050EAF
:1029A000DBCF01F0060EDBCF02F0070EDBCF03F02A
:1029B000005001100210031001E128D10E0EDBCFF0
:1029C00000F0016A026A036AD950040FE96E000E32
:1029D000DA20EA6EEE500026EE500122EE5002227E
:1029E000EE500322110EDBCFE9FF120EDBCFEAFF20
:1029F000260EE926000EEA2200C0EEFF01C0EEFF1F
:102A000002C0EEFF03C0EEFF110EDBCFE9FF120E96
:102A1000DBCFEAFF260EE926000EEA22EECFE6FF24
:102A2000EECFE6FFEECFE6FFEFCFE6FFE66EE66A1B
:102A300065EC4CF0006E060EE15C02E2E16AE552E4
:102A4000E16E0050000901E0E1D0110EDBCFE9FF9B
:102A5000120EDBCFEAFFEE52EF8C110EDBCFE9FF57
:102A6000120EDBCFEAFF160EE926000EEA22EECFA9
:102A700000F0EFCF01F00001010E0116000ED8802A
:102A80000056020E01560F0E00C0DBFF100E01C0F3
:102A9000DBFF0F0EDBCF00F0100EDBCF01F0FA0EE4
:102AA000DBCF02F0FB0EDBCF03F00050025C0150E5
:102AB00003580CE2FA0EDBCF3FF0FB0EDBCF40F009
:102AC0000F0E3FC0DBFF100E40C0DBFF0F0EDBCF51
:102AD00000F0100EDBCF01F0026A036A00C0E6FFCF
:102AE00001C0E6FF02C0E6FF03C0E6FF0C0EDBCF2D
:102AF000E6FF0D0EDBCFE6FF65EC4CF0046E060E34
:102B0000E15C02E2E16AE552E16E0450000901E095
:102B10007DD00F0EDBCF00F0100EDBCF01F0026A8C
:102B2000036A110EDBCFE9FF120EDBCFEAFF160EB0
:102B3000E926000EEA220050EE260150EE22025055
:102B4000EE220350EE220F0EDBCF00F0100EDBCF93
:102B500001F0D9500C0FE96E000EDA20EA6E005039
:102B6000EE260150ED220F0EDBCF00F0100EDBCF72
:102B700001F0D950FA0FE96EFF0EDA20EA6E00502C
:102B8000EE5E0150ED5A0F0EDBCF00F0100EDBCFE2
:102B900001F0F80EDBCFE9FFF90EDBCFEAFF0050C2
:102BA000EE260150ED22110EDBCFE9FF120EDBCF36
:102BB000EAFF160EE926000EEA22EECF00F0EFCF74
:102BC00001F00001010E01160050011001E0F1D5E5
:102BD000E66AE66AE66AE66A000EE66EE66A65ECB2
:102BE0004CF0006E060EE15C02E2E16AE552E16E35
:102BF000005000090BE1110EDBCFE9FF120EDBCF15
:102C0000EAFFEE52EF9CD5D5000E09D0110EDBCFB6
:102C1000E9FF120EDBCFEAFFEE52EF6A010E006E03
:102C2000130EE15C02E2E16AE552E16E0050E5520A
:102C3000E5CFDAFFE7CFD9FF1200D9CFE6FFDACF31
:102C4000E6FFE1CFD9FFE2CFDAFF120EE12402E383
:102C5000E168E652E16E100EFEC4DBFF110EFFC408
:102C6000DBFFD950100FE96E000EDA20EA6EEE504D
:102C7000ED1002E1060EEDD2100EDBCFE9FF110ED2
:102C8000DBCFEAFFEE52EF50010B02E1050EE1D27D
:102C9000FA0EDBCF00F0FB0EDBCF01F0FC0EDBCF3A
:102CA00002F0FD0EDBCF03F0100EDBCFE9FF110EBB
:102CB000DBCFEAFF1A0EE926000EEA220050EE5C96
:102CC0000150EE580250EE580350EE5816E2100E26
:102CD000DBCFE9FF110EDBCFEAFF1A0EE926000E6B
:102CE000EA22FA0EEECFDBFFFB0EEECFDBFFFC0E8F
:102CF000EECFDBFFFD0EEECFDBFF100EDBCFE9FFEB
:102D0000110EDBCFEAFF160EE926000EEA220C0EAA
:102D1000EECFDBFF0D0EEECFDBFF0E0EEECFDBFFB7
:102D20000F0EEECFDBFF100EDBCFE9FF110EDBCF76
:102D3000EAFF160EE926000EEA22EE6AEE6AEE6A55
:102D4000EE6AD950FA0FE96EFF0EDA20EA6ED880EB
:102D5000000EEE54000EEE54000EEE54000EEE5433
:102D600001E36CD2100EDBCFE9FF110EDBCFEAFFDF
:102D7000020EE926000EEA22EFCF3DF03E6A3F6ADE
:102D8000406A426A020E436E446A456A22EC57F07A
:102D9000040E39C0DBFF050E3AC0DBFF060E3BC058
:102DA000DBFF070E3CC0DBFFD9500C0FE96E000EB5
:102DB000DA20EA6ED880000EEE54000EEE54000EBB
:102DC000EE54000EEE5401E3D5D00C0EDBCF08F02C
:102DD0000D0EDBCF09F00E0EDBCF0AF00F0EDBCFAE
:102DE0000BF00806000E095A0A5A0B5A08C03DF0AB
:102DF00009C03EF00AC03FF00BC040F0040EDBCF2C
:102E000042F0050EDBCF43F0060EDBCF44F0070E99
:102E1000DBCF45F087EC57F03DC004F03EC005F035
:102E20003FC006F040C007F0FA0EDBCF00F0FB0E0B
:102E3000DBCF01F0FC0EDBCF02F0FD0EDBCF03F0A9
:102E40000006000E015A025A035A00C03DF001C0AC
:102E50003EF002C03FF003C040F0040EDBCF42F072
:102E6000050EDBCF43F0060EDBCF44F0070EDBCFC1
:102E700045F087EC57F004503D5C05503E58065035
:102E80003F580750405876E30C0EDBCF00F00D0E94
:102E9000DBCF01F00E0EDBCF02F00F0EDBCF03F025
:102EA0000006000E015A025A035A040EDBCF04F04A
:102EB000050EDBCF05F0060EDBCF06F0070EDBCFED
:102EC00007F00406000E055A065A075A041E051E8E
:102ED000061E071E04500016055001160650021665
:102EE00007500316100EDBCFE9FF110EDBCFEAFF10
:102EF000160EE926000EEA2200C0EEFF01C0EEFF2A
:102F000002C0EEFF03C0EEFF100EDBCFE9FF110E93
:102F1000DBCFEAFF160EE926000EEA22EECF00F024
:102F2000EECF01F0EECF02F0EFCF03F0D950FA0F61
:102F3000E96EFF0EDA20EA6E0050EE5E0150EE5AA6
:102F40000250EE5A0350EE5A100EDBCFE9FF110E7D
:102F5000DBCFEAFF220EE926000EEA22EECFDFFFEA
:102F6000010EEECFDBFF020EEECFDBFF030EEECF46
:102F7000DBFF2AD0100EDBCFE9FF110EDBCFEAFF1B
:102F80001E0EE926000EEA22EECFDFFF010EEECF85
:102F9000DBFF020EEECFDBFF030EEECFDBFF100EEA
:102FA000DBCFE9FF110EDBCFEAFF220EE926000E90
:102FB000EA22DFCFEEFF010EDBCFEEFF020EDBCF0A
:102FC000EEFF030EDBCFEEFF040EDBCF00F0050EAD
:102FD000DBCF01F0060EDBCF02F0070EDBCF03F0F4
:102FE000D950FA0FE96EFF0EDA20EA6EEE50005C5F
:102FF000EE500158EE500258EE50035801E389D0CC
:10300000D9CFE9FFDACFEAFFEECFE6FFEECFE6FF5A
:10301000EECFE6FFEFCFE6FFB2EC00F0E552E5526F
:10302000E552E5523DC0DEFF3EC0DEFF3FC0DEFFA1
:1030300040C0DDFFDD52DD52D9CFE9FFDACFEAFF34
:10304000D880010EEE54000EEE54000EEE54000E29
:10305000EE5401E3F5D0100EDBCFE9FF110EDBCF0C
:10306000EAFF060EE926000EEA22EECF00F0EECFD0
:1030700001F0EECF02F0EFCF03F0D9CFE9FFDACFC6
:10308000EAFF0050EE5C0150EE580250EE5803503B
:10309000EE5801E3D5D0100EDBCFE9FF110EDBCFE8
:1030A000EAFF220EE926000EEA22DFCFEEFF010E34
:1030B000DBCFEEFF020EDBCFEEFF030EDBCFEEFF2A
:1030C000100EDBCFE9FF110EDBCFEAFF160EE9266B
:1030D000000EEA22040EDB50EE26050EDB50EE2237
:1030E000060EDB50EE22070EDB50EE22D950FA0F0F
:1030F000E96EFF0EDA20EA6E040EDB50EE5E050E7E
:10310000DB50EE5A060EDB50EE5A070EDB50EE5A3D
:103110005BD7100EDBCFE9FF110EDBCFEAFF160EF7
:10312000E926000EEA22FA0EDB50EE26FB0EDB50FB
:10313000EE22FC0EDB50EE22FD0EDB50EE22D9CF4C
:10314000E9FFDACFEAFFEECFE6FFEECFE6FFEECF04
:10315000E6FFEFCFE6FF66EC03F0E552E552E552FD
:10316000E552080E3DC0DBFF090E3EC0DBFF0A0E34
:103170003FC0DBFF0B0E40C0DBFF080EDBCF00F0D3
:10318000090EDBCF01F00A0EDBCF02F00B0EDBCF16
:1031900003F0005001100210031052E0100EDBCFBC
:1031A000E9FF110EDBCFEAFF160EE926000EEA2238
:1031B000EECF00F0EECF01F0EECF02F0EFCF03F054
:1031C000090ED8900332023201320032E806F9E1EA
:1031D000100EDBCFE9FF110EDBCFEAFF020EE9266E
:1031E000000EEA22EF04056A066A076AE850001634
:1031F000055001160650021607500316D950080F45
:10320000E96E000EDA20EA6EEE500026EE50012242
:10321000EE500222EE500322100EDBCFE9FF110E1A
:10322000DBCFEAFF260EE926000EEA2200C0EEFF01
:1032300001C0EEFF02C0EEFF03C0EEFF000E09D09A
:10324000100EDBCFE9FF110EDBCFEAFFEE52EF6A83
:10325000010E006E120EE15C02E2E16AE552E16EDF
:0E3260000050E552E5CFDAFFE7CFD9FF1200AC
:02326E000F014E
:10327000006B016B086B096B0A6B0B6BA4C400F04D
:10328000016A026A036A000E006C011E0122021E1E
:103290000222031E0322A5C404F0056A066A076A17
:1032A000180ED8900436053606360736E806F9E1DA
:1032B0000450002605500122065002220750032226
:1032C000A6C408F0096A0A6A0B6A100ED89008367C
:1032D00009360A360B36E806F9E10850002609508F
:1032E00001220A5002220B500322A7C43DF03E6A7D
:1032F0003F6A406A426A010E436E446A456A22ECA4
:1033000057F0005039240F010C6F01503A200D6F17
:1033100002503B200E6F03503C200F6F0CCFE6FF96
:103320000DCFE6FF0ECFE6FFE66E0CCFE6FF0DCF2A
:10333000E6FF0ECFE6FFE66EAD0E006EA10E016E4B
:10334000026A00C0E6FFE66E02C0E6FF800EE66E8F
:10335000000EE66E3BEC56F0036E0D0EE15C02E2F1
:10336000E16AE552E16E0350800EE66E000EE66EF5
:1033700087EC54F0E552E552306A316A326A336ABA
:10338000346A356A020E366E0F01146B8090A70EF8
:10339000006EA10E016E026A00C0E6FFE66E02C07A
:1033A000E6FF800EE66E000EE66E3BEC56F0036E16
:1033B000050EE15C02E2E16AE552E16E0350800E27
:1033C000E66E000EE66E87EC54F0E552E552120010
:1033D000D9CFE6FFDACFE6FFE1CFD9FFE2CFDAFFC0
:1033E000E652FB0EDB5001E042DFDF6AFC0EDB50F1
:1033F00007E0FD0EDB507F0BE76EFD0EE7CFDBFF36
:10340000FC0EDB5001E1E3D0FD0EDB50040804E0CC
:10341000FD0EDB50140803E1070EDF6E11D2FD0E26
:10342000DB503F0802E1316A17D0FD0EDB505F0828
:1034300002E1306A11D0400EF36EFD0EDBCFF4FFD7
:10344000F350F45C0BE3FD0EDB505E0807E3FD0E6A
:10345000DB50400803E0306A336AB6D0FD0EDB5023
:10346000400818E1010E306E336AA10E006EA10E05
:10347000016E026A00C0E6FFE66E02C0E6FF800E43
:10348000E66E000EE66E3BEC56F0036E050EE15C58
:103490001EE21BD0FD0EDB50200824E1010E316E30
:1034A000336A9B0E006EA10E016E026A00C0E6FF39
:1034B000E66E02C0E6FF800EE66E000EE66E3BECA6
:1034C00056F0036E050EE15C02E2E16AE552E16E40
:1034D0000350800EE66E000EE66E87EC54F0E55267
:1034E000E55272D0FD0EDB50650806E1315004E074
:1034F000346A356A010E67D0FD0EDB506E0802E1BA
:10350000020E336EFD0EDB50700806E1305004E011
:10351000346A356A030E336EFD0EDB50700827E106
:10352000315025E08080950E006EA10E016E026A7A
:1035300000C0E6FFE66E02C0E6FF800EE66E000EFB
:10354000E66E3BEC56F0036E050EE15C02E2E16ACA
:10355000E552E16E0350800EE66E000EE66E87ECDB
:1035600054F0E552E552346A356A040E2CD0FD0E53
:10357000DB5072082CE131502AE08080950E006EFD
:10358000A10E016E026A00C0E6FFE66E02C0E6FF11
:10359000800EE66E000EE66E3BEC56F0036E050EF6
:1035A000E15C02E2E16AE552E16E0350800EE66EF4
:1035B000000EE66E87EC54F0E552E5522A0E346EAA
:1035C0001C0E356E050E336EF36AF46A41D133502A
:1035D000050A01E1EAD0010A01E1A0D0070A36E0BC
:1035E000010A0AE0030A02E0010A2DD1FD0EDBCF39
:1035F000E6FF35D9E55290D08080950E006EA10E81
:10360000016E026A00C0E6FFE66E02C0E6FF800EB1
:10361000E66E000EE66E3BEC56F0036E050EE15CC6
:1036200002E2E16AE552E16E0350800EE66E000EA2
:10363000E66E87EC54F0E552E552FD0EDBCFE6FF77
:10364000B8EC1FF0E552DF6E336AFDD08080950E36
:10365000006EA10E016E026A00C0E6FFE66E02C0B7
:10366000E6FF800EE66E000EE66E3BEC56F0036E53
:10367000050EE15C02E2E16AE552E16E0350800E64
:10368000E66E000EE66E87EC54F0E552E5523650D9
:10369000E66EE66A800E006EA10E016E026A00C040
:1036A000E6FFE66E02C0E6FF800EE66E000EE66EF6
:1036B0003BEC56F0036E070EE15C02E2E16AE55274
:1036C000E16E0350800EE66E000EE66E87EC54F05D
:1036D000E552E552E66A010EE66EE66A000EE66E17
:1036E000020EE66EF8EC54F0006E050EE15C02E2AC
:1036F000E16AE552E16E0050020E1E101E6E36C0E9
:1037000000F2010EE66EE66A1AEC51F0E552E5525F
:10371000FD0E1E141E6E080EDF6E95D08090A70E53
:10372000006EA10E016E026A00C0E6FFE66E02C0E6
:10373000E6FF800EE66E000EE66E3BEC56F0036E82
:10374000050EE15C02E2E16AE552E16E0350800E93
:10375000E66E000EE66E87EC54F0E552E552DF6A45
:10376000FD0EDBCFE6FFE66A690E006EA10E016E6C
:10377000026A00C0E6FFE66E02C0E6FF800EE66E5B
:10378000000EE66E3BEC56F0036E070EE15C02E2C3
:10379000E16AE552E16E0350800EE66E000EE66EC1
:1037A00087EC54F0E552E5524ED0FD0EDB50080890
:1037B0004AE1FD0EDBCFE6FFE66A510E006EA10E78
:1037C000016E026A00C0E6FFE66E02C0E6FF800EF0
:1037D000E66E000EE66E3BEC56F0036E070EE15C03
:1037E00002E2E16AE552E16E0350800EE66E000EE1
:1037F000E66E87EC54F0E552E5528090A70E006E1D
:10380000A10E016E026A00C0E6FFE66E02C0E6FF8E
:10381000800EE66E000EE66E3BEC56F0036E050E73
:10382000E15C02E2E16AE552E16E0350800EE66E71
:10383000000EE66E87EC54F0E552E552DF6A366A18
:10384000336A346A356ADF50016AF36E01C0F4FFEF
:10385000E552E552E5CFDAFFE7CFD9FF1200D9CF25
:10386000E6FFDACFE6FFE1CFD9FFE2CFDAFFE6529B
:10387000DF6A2A0E341802E11C0E351801E170D3FC
:103880000F0E341802E1270E351801E169D3760EC8
:10389000341802E10E0E351801E11ED3750E3418EE
:1038A00002E10E0E351801E112D3AC0E341802E11C
:1038B0000D0E351801E154D3480E341802E10D0EF7
:1038C000351801E1E1D20C0E341802E1070E35186B
:1038D00001E197D20B0E341802E1070E351801E111
:1038E00089D20A0E341802E1070E351801E17DD2A3
:1038F000090E341802E1070E351801E171D2EE0EFF
:10390000341802E1030E351801E1FBD1ED0E341835
:1039100002E1030E351801E1EDD1EC0E341802E19D
:10392000030E351801E1E1D1EB0E341802E1030E6C
:10393000351801E1D5D1EA0E341802E1030E35182D
:1039400001E1C9D1E90E341802E1030E351801E195
:10395000BDD1345001E004D3355001E001D3FD0E58
:10396000DB503DE131503BE0450E006EA10E016E93
:10397000026A00C0E6FFE66E02C0E6FF800EE66E59
:10398000000EE66E3BEC56F0036E050EE15C02E2C3
:10399000E16AE552E16E0350800EE66E000EE66EBF
:1039A00087EC54F0E552E552DF6A0A0E346E356A50
:1039B0008090A70E006EA10E016E026A00C0E6FFA5
:1039C000E66E02C0E6FF800EE66E000EE66E3BEC91
:1039D00056F0036E050EE15C01E3B8D2B5D2FD0EE0
:1039E000DB5002083DE131503BE0380E006EA10E85
:1039F000016E026A00C0E6FFE66E02C0E6FF800EBE
:103A0000E66E000EE66E3BEC56F0036E050EE15CD2
:103A100002E2E16AE552E16E0350800EE66E000EAE
:103A2000E66E87EC54F0E552E552DF6A140E346E10
:103A3000356A8090A70E006EA10E016E026A00C06A
:103A4000E6FFE66E02C0E6FF800EE66E000EE66E52
:103A50003BEC56F0036E050EE15C01E377D274D2C5
:103A6000200EF36EFD0EDBCFF4FFF350F45C48E361
:103A7000FD0EDB502F0844E3315042E0FD0EDB50D9
:103A8000E00F0F01006FE850E66EE66A250E006E4B
:103A9000A10E016E026A00C0E6FFE66E02C0E6FFFC
:103AA000800EE66E000EE66E3BEC56F0036E070EDF
:103AB000E15C02E2E16AE552E16E0350800EE66EDF
:103AC000000EE66E87EC54F0E552E552DF6A346A88
:103AD000356A8090A70E006EA10E016E026A00C0CA
:103AE000E6FFE66E02C0E6FF800EE66E000EE66EB2
:103AF0003BEC56F0036E050EE15C01E327D224D2C5
:103B0000400EF36EFD0EDBCFF4FFF350F45C30E3B8
:103B1000FD0EDB504F082CE331502AE0FD0EDB5048
:103B2000C00F0F01016FE850E66EE66A100E006EDE
:103B3000A10E016E026A00C0E6FFE66E02C0E6FF5B
:103B4000800EE66E000EE66E3BEC56F0036E070E3E
:103B5000E15C02E2E16AE552E16E0350800EE66E3E
:103B6000000EE66E87EC54F0E552E552DF6AACD108
:103B7000FD0EDB5035083EE131503CE0000E006E9A
:103B8000A10E016E026A00C0E6FFE66E02C0E6FF0B
:103B9000800EE66E000EE66E3BEC56F0036E050EF0
:103BA000E15C02E2E16AE552E16E0350800EE66EEE
:103BB000000EE66E87EC54F0E552E552DF6AAC0E7B
:103BC000346E0D0E356E8090A70E006EA10E016E44
:103BD000026A00C0E6FFE66E02C0E6FF800EE66EF7
:103BE000000EE66E3BEC56F0036E050EE15C01E361
:103BF000ADD1AAD1FD0EDB500D083EE131503CE0C5
:103C0000DF6ABC0E346E020E356E8090A70E006E19
:103C1000A10E016E026A00C0E6FFE66E02C0E6FF7A
:103C2000800EE66E000EE66E3BEC56F0036E050E5F
:103C3000E15C02E2E16AE552E16E0350800EE66E5D
:103C4000000EE66E87EC54F0E552E552EE0E006E83
:103C5000A00E016E026A00C0E6FFE66E02C0E6FF3B
:103C6000800EE66E000EE66E3BEC56F0036E050E1F
:103C7000E15C01E36BD168D1FD0EDB50100804E17B
:103C8000315002E0E90E3AD0FD0EDB50180804E195
:103C9000315002E0090EB2D0FD0EDBCFE6FFE66A3E
:103CA000DB0E006EA00E016E026A00C0E6FFE66E3B
:103CB00002C0E6FF800EE66E000EE66E3BEC56F0AC
:103CC000036E070EE15C01E341D13ED1FD0EDBCF77
:103CD00002FFEA0E13D0FD0EDBCF03FFEB0E0ED07A
:103CE000FD0EDBCF04FFEC0E09D0FD0EDBCF05FF90
:103CF000ED0E04D0FD0EDBCF06FFEE0E346E030E8C
:103D0000E9D0FD0EDBCF07FF04CF00F0016A026AA5
:103D1000036A000E006C011E0122021E0222031E15
:103D2000032205CF04F0056A066A076A180ED890C8
:103D30000436053606360736E806F9E10450002653
:103D400005500122065002220750032206CF08F038
:103D5000096A0A6A0B6A100ED890083609360A36C4
:103D60000B36E806F9E108500026095001220A50F6
:103D700002220B50032207CF3DF03E6A3F6A406AA1
:103D8000426A010E436E446A456A22EC57F00050C5
:103D900039240F01086F01503A20096F02503B206F
:103DA0000A6F03503C200B6F08CFE6FF09CFE6FFF8
:103DB0000ACFE6FFE66EC30E006EA00E016E026A29
:103DC00000C0E6FFE66E02C0E6FF800EE66E000E63
:103DD000E66E3BEC56F0036E090EE15C6BE268D0D8
:103DE000FD0EDBCF13FF0A0E09D0FD0EDBCF12FF55
:103DF0000B0E04D0FD0EDBCF11FF0C0E346E070E40
:103E000069D0FD0EDBCF10FF10CFE6FF11CFE6FF2C
:103E100012CFE6FF13CFE6FFAC0E006EA00E016ED0
:103E2000026A00C0E6FFE66E02C0E6FF800EE66EA4
:103E3000000EE66E3BEC56F0036E090EE15C02E20A
:103E4000E16AE552E16E0350800EE66E000EE66E0A
:103E500087EC54F0E552E552346A356A8090A70E3B
:103E6000006EA10E016E026A00C0E6FFE66E02C09F
:103E7000E6FF800EE66E000EE66E3BEC56F0036E3B
:103E8000050EE15C63E260D0A10E006EA00E016E33
:103E9000026A00C0E6FFE66E02C0E6FF800EE66E34
:103EA000000EE66E3BEC56F0036E050EE15C02E29E
:103EB000E16AE552E16E0350800EE66E000EE66E9A
:103EC00087EC54F0E552E552346A356A49D0760EF3
:103ED000346E0E0E356E44D0900E006EA00E016E44
:103EE000026A00C0E6FFE66E02C0E6FF800EE66EE4
:103EF000000EE66E3BEC56F0036E050EE15C02E24E
:103F0000E16AE552E16E0350800EE66E000EE66E49
:103F100087EC54F0E552E552346A356ADF6A8090E6
:103F2000A70E006EA10E016E026A00C0E6FFE66EEB
:103F300002C0E6FF800EE66E000EE66E3BEC56F029
:103F4000036E050EE15C02E2E16AE552E16E0350A8
:103F5000800EE66E000EE66E87EC54F0E552E552F8
:103F6000DF50E552E552E5CFDAFFE7CFD9FF120087
:103F7000D9CFE6FFDACFE6FFE1CFD9FFE2CFDAFF14
:103F8000E6520F0E341802E1270E351823E0BC0E5E
:103F9000341802E1020E351819E0AC0E341802E1B3
:103FA0000D0E351811E0140E341801E1355007E0FC
:103FB0000A0E34180EE135500CE1030E08D0050E40
:103FC000DF6E346A356A06D0010E01D0020EDF6E54
:103FD00001D0DF6ADF50E552E552E5CFDAFFE7CFE7
:103FE000D9FF12007E0E006EA00E016E026A00C0A4
:103FF000E6FFE66E02C0E6FF800EE66E000EE66E9D
:104000003BEC56F0036E050EE15C02E2E16AE5521C
:10401000E16E0350800EE66E000EE66E87EC54F003
:10402000E552E552FD0E1E141E6E050EE66EE66AA2
:10403000840EE66E040EE66E000EE66E020EE66E6E
:10404000CDEC54F0006E060EE15C02E2E16AE5524E
:10405000E16E0050050EE66EE66A1AEC51F0E5528C
:10406000E552130EE66EE66A890EE66E040EE66E03
:10407000000EE66E020EE66ECDEC54F0006E060EFB
:10408000E15C02E2E16AE552E16E0050130EE66E79
:10409000E66A1AEC51F0E552E552020E1E101E6E51
:1040A0000D0EE66EE66A9C0EE66E040EE66E000EDF
:1040B000E66E020EE66ECDEC54F0006E060EE15C8C
:1040C00002E2E16AE552E16E00500D0EE66EE66A2C
:1040D0001AEC51F0E552E552FD0E1E141E6E809052
:1040E000A70E006EA10E016E026A00C0E6FFE66E2A
:1040F00002C0E6FF800EE66E000EE66E3BEC56F068
:10410000036E050EE15C02E2E16AE552E16E0350E6
:10411000800EE66E000EE66E87EC54F0E552E55236
:1041200012006E0E006EA00E016E026A00C0E6FF65
:10413000E66E02C0E6FF800EE66E000EE66E3BEC19
:1041400056F0036E050EE15C02E2E16AE552E16EB3
:104150000350800EE66E000EE66E87EC54F0E552DA
:10416000E552020E1E101E6EE66A010EE66EE66A4B
:10417000000EE66E020EE66EF8EC54F0006E050ED0
:10418000E15C02E2E16AE552E16E00500201110ECB
:10419000006F01690F0114A503D00201010E046F25
:1041A0000F0114A103D00201020E066F0F0114A328
:1041B00003D00201020E066F82A403D00201080E92
:1041C000066F14CF36F002CF0BF203CF0CF204CF00
:1041D0000DF205CF0EF206CF0FF207CF10F2140E3C
:1041E000E66EE66A1AEC51F0E552E552FD0E1E1439
:1041F0001E6E8090A70E006EA10E016E026A00C0B6
:10420000E6FFE66E02C0E6FF800EE66E000EE66E8A
:104210003BEC56F0036E050EE15C02E2E16AE5520A
:10422000E16E0350800EE66E000EE66E87EC54F0F1
:10423000E552E5521200D9CFE6FFDACFE6FFE1CF33
:10424000D9FFE2CFDAFFE652E652E652E652E652F4
:1042500008CFDFFF010E09CFDBFF020E0ACFDBFF25
:10426000030E0BCFDBFF5F0E006EA00E016E026A25
:1042700000C0E6FFE66E02C0E6FF800EE66E000EAE
:10428000E66E3BEC56F0036E050EE15C02E2E16A7D
:10429000E552E16E0350800EE66E000EE66E87EC8E
:1042A00054F0E552E552D9CFE9FFDACFEAFFEECF7D
:1042B000E6FFEECFE6FFEECFE6FFEFCFE6FFD9CF8A
:1042C000E9FFDACFEAFFEECFE6FFEECFE6FFEECF73
:1042D000E6FFEFCFE6FF470E006EA00E016E026A0A
:1042E00000C0E6FFE66E02C0E6FF800EE66E000E3E
:1042F000E66E3BEC56F0036E0D0EE15C02E2E16A05
:10430000E552E16E0350800EE66E000EE66E87EC1D
:1043100054F0E552E552080EE96E0F0EEA6EEE50CB
:104320000F010C5DEE500D59EE500E59EE500F5925
:1043300026E2350E006EA00E016E026A00C0E6FF96
:10434000E66E02C0E6FF800EE66E000EE66E3BEC07
:1043500056F0036E050EE15C02E2E16AE552E16EA1
:104360000350800EE66E000EE66E87EC54F0E552C8
:10437000E552010E366E040E0F011411146F100E6B
:10438000E96E0F0EEA6E0851EE24006E0951EE2020
:10439000016E0A51EE20026E0B51EE20036E0050AA
:1043A0000C5D01500D5902500E5903500F5926E271
:1043B000230E006EA00E016E026A00C0E6FFE66EDC
:1043C00002C0E6FF800EE66E000EE66E3BEC56F095
:1043D000036E050EE15C02E2E16AE552E16E035014
:1043E000800EE66E000EE66E87EC54F0E552E55264
:1043F000010E366E040E0F011411146F366AD9CFF8
:10440000E9FFDACFEAFFEECFE6FFEECFE6FFEECF31
:10441000E6FFEFCFE6FF1DEC16F0E552E552E55260
:10442000E552E76E040EE7CFDBFFDB503CE0040E05
:10443000DBCF00F0016A00BE016800C0E6FF01C0EA
:10444000E6FFD9CFE9FFDACFEAFFEECFE6FFEECF06
:10445000E6FFEECFE6FFEFCFE6FF0B0E026EA00EFB
:10446000036E046A02C0E6FFE66E04C0E6FF800E3B
:10447000E66E000EE66E3BEC56F0056E0B0EE15C50
:1044800002E2E16AE552E16E0550800EE66E000E32
:10449000E66E87EC54F0E552E552010E366E040EDE
:1044A0000F011411146F3650006E016A36C0F3FF0D
:1044B00001C0F4FF050EE15C02E2E16AE552E16E43
:1044C000E552E5CFDAFFE7CFD9FF1200D9CFE6FFFB
:1044D000DACFE6FFE1CFD9FFE2CFDAFF0F0EE1241A
:1044E00002E3E168E652E16E8080950E006EA10E57
:1044F000016E026A00C0E6FFE66E02C0E6FF800EB3
:10450000E66E000EE66E3BEC56F0036E050EE15CC7
:1045100002E2E16AE552E16E0350800EE66E000EA3
:10452000E66E87EC54F0E552E55208CFE6FF09CF7E
:10453000E6FF0ACFE6FF0BCFE6FF08CFE6FF09CF85
:10454000E6FF0ACFE6FF0BCFE6FFF30E006E9F0EED
:10455000016E026A00C0E6FFE66E02C0E6FF800E52
:10456000E66E000EE66E3BEC56F0036E0D0EE15C5F
:1045700002E2E16AE552E16E0350800EE66E000E43
:10458000E66E87EC54F0E552E55255DE020EF3CFAD
:10459000DBFF030EF4CFDBFFD950020FE96E000EF4
:1045A000DA20EA6EEE50ED1001E07FD110CF3DF041
:1045B00011CF3EF012CF3FF013CF40F0426A010E10
:1045C000436E446A456A87EC57F00B0E3DC0DBFF33
:1045D0000C0E3EC0DBFF10CF3DF011CF3EF012CFEE
:1045E0003FF013CF40F0426A010E436E446A456AC1
:1045F00087EC57F00D0E39C0DBFF0E0E3AC0DBFF23
:10460000FD0E1E141E6E040EDB6A050EDB6A060E1E
:10461000DB6A070EDB6ADE6ADD6ADECF00F0DDCF23
:1046200001F00B0EDBCF02F00C0EDBCF03F00150DC
:104630000318E8AE02D0033404D00250005C0350EB
:10464000015801E3D2D00B0EDBCF00F00C0EDBCF14
:1046500001F00006000E015A0050DF1810E1015071
:10466000DE52DD180CE1D9500D0FE96E000EDA2094
:10467000EA6EEE50ED1003E1020E1E101E6ED950D0
:10468000090FE66E000EDA20E66EE66A010EE66EAF
:10469000000EE66E020EE66E35EC10F0006E060EB1
:1046A000E15C02E2E16AE552E16E0050E76E080E5D
:1046B000E7CFDBFF090EDBCFE6FF0A0EDBCFE6FF1D
:1046C000080EDBCF00F0016A00BE016800C0E6FF03
:1046D00001C0E6FFD90E026E9F0E036E046A02C08F
:1046E000E6FFE66E04C0E6FF800EE66E000EE66EA4
:1046F0003BEC56F0056E090EE15C02E2E16AE55220
:10470000E16E0550800EE66E000EE66E87EC54F00A
:10471000E552E552080EDB5001E0C7D0090EDBCFB1
:10472000E6FF0A0EDBCFE6FF1AEC51F0E552E55248
:10473000090EDBCF00F00A0EDBCF01F0026A036A3C
:10474000D950040FE96E000EDA20EA6EEE50002612
:10475000EE500122EE500222EE500322040E00C061
:10476000DBFF050E01C0DBFF060E02C0DBFF070EFC
:1047700003C0DBFF0F01092B000E0A230B2308CF18
:10478000E6FF09CFE6FF0ACFE6FF0BCFE6FF08CF33
:10479000E6FF09CFE6FF0ACFE6FF0BCFE6FFC50E27
:1047A000006E9F0E016E026A00C0E6FFE66E02C058
:1047B000E6FF800EE66E000EE66E3BEC56F0036EF2
:1047C0000D0EE15C02E2E16AE552E16E0350800EFB
:1047D000E66E000EE66E87EC54F0E552E552DF2AF5
:1047E000010E01E21AD7DB2A18D70D0EDBCF00F03D
:1047F0000E0EDBCF01F0013401E3C8D000500008F9
:10480000000E015401E3C2D0D950090FE66E000E2C
:10481000DA20E66E0D0EDBCFE6FF0E0EDBCFE6FFF5
:10482000000EE66E020EE66E35EC10F0006E060E1F
:10483000E15C02E2E16AE552E16E0050E76E080ECB
:10484000E7CFDBFF090EDBCFE6FF0A0EDBCFE6FF8B
:10485000080EDBCF00F0016A00BE016800C0E6FF71
:1048600001C0E6FFAB0E026E9F0E036E046A02C02B
:10487000E6FFE66E04C0E6FF800EE66E000EE66E12
:104880003BEC56F0056E090EE15C02E2E16AE5528E
:10489000E16E0550800EE66E000EE66E87EC54F079
:1048A000E552E552080EDB500DE0040E0F01141125
:1048B000146FECEC2BF0020EDBCF00F0030EDBCF1D
:1048C00001F0BAD0020E1E101E6E0D0EDBCFE6FFF9
:1048D0000E0EDBCFE6FF1AEC51F0E552E552090E61
:1048E000DBCF00F00A0EDBCF01F0026A036AD95079
:1048F000040FE96E000EDA20EA6EEE500026EE504C
:104900000122EE500222EE500322040E00C0DBFF13
:10491000050E01C0DBFF060E02C0DBFF070E03C061
:10492000DBFF0F01092B000E0A230B2308CFE6FF44
:1049300009CFE6FF0ACFE6FF0BCFE6FF08CFE6FF81
:1049400009CFE6FF0ACFE6FF0BCFE6FFC50E006EEC
:104950009F0E016E026A00C0E6FFE66E02C0E6FF2F
:10496000800EE66E000EE66E3BEC56F0036E0D0E0A
:10497000E15C02E2E16AE552E16E0350800EE66E10
:10498000000EE66E87EC54F0E552E552FD0E1E1463
:104990001E6ED950040FE96E000EDA20EA6EEECFDB
:1049A000E6FFEECFE6FFEECFE6FFEFCFE6FF980E95
:1049B000006E9F0E016E026A00C0E6FFE66E02C046
:1049C000E6FF800EE66E000EE66E3BEC56F0036EE0
:1049D000090EE15C02E2E16AE552E16E0350800EED
:1049E000E66E000EE66E87EC54F0E552E552366A4C
:1049F0008090A70E006EA10E016E026A00C0E6FF55
:104A0000E66E02C0E6FF800EE66E000EE66E3BEC40
:104A100056F0036E050EE15C02E2E16AE552E16EDA
:104A20000350800EE66E000EE66E87EC54F0E55201
:104A3000E5523650006E016A00C0F3FF01C0F4FF7A
:104A40000F0EE15C02E2E16AE552E16EE552E5CF6C
:104A5000DAFFE7CFD9FF1200D9CFE6FFDACFE6FFC2
:104A6000E1CFD9FFE2CFDAFF0F0EE12402E3E168E4
:104A7000E652E16E366A08CFE6FF09CFE6FF0ACFBD
:104A8000E6FF0BCFE6FF08CFE6FF09CFE6FF0ACF30
:104A9000E6FF0BCFE6FF7F0E006E9F0E016E026AEF
:104AA00000C0E6FFE66E02C0E6FF800EE66E000E76
:104AB000E66E3BEC56F0036E0D0EE15C02E2E16A3D
:104AC000E552E16E0350800EE66E000EE66E87EC56
:104AD00054F0E552E5521BEC21F00B0EF3CFDBFF57
:104AE0000C0EF4CFDBFFD9500B0FE96E000EDA206D
:104AF000EA6EEE50ED1007E00B0EDBCF00F00C0E6F
:104B0000DBCF01F0FFD0060EDB6A070EDB6A080E72
:104B1000DB6A090EDB6A010EDE6EDD6AD9CFE9FFC2
:104B2000DACFEAFFEE50ED1001E1F1D00001AD6BFC
:104B3000AE6B4FEC52F00B0EF3CFDBFF0C0EF4CF4D
:104B4000DBFF0001000ED880AD55000EAE552AE205
:104B5000ADC0E6FFAEC0E6FF0B0EDBCFE6FF0C0EEE
:104B6000DBCFE6FF670E006E9F0E016E026A00C08B
:104B7000E6FFE66E02C0E6FF800EE66E000EE66E11
:104B80003BEC56F0036E090EE15C02E2E16AE5528D
:104B9000E16E0350800EE66E000EE66E87EC54F078
:104BA000E552E552ADC000F0AEC001F0026A036A02
:104BB000D950060FE96E000EDA20EA6EEE5000269C
:104BC000EE500122EE500222EE500322060E00C0EB
:104BD000DBFF070E01C0DBFF080E02C0DBFF090E82
:104BE00003C0DBFFD950060FE96E000EDA20EA6E33
:104BF0000F011051EE5C1151EE581251EE58135145
:104C0000EE5802E3DE6ADD6AD9500B0FE96E000E42
:104C1000DA20EA6EFE0EEE1804E1ED5002E1DE6AE3
:104C2000DD6A81BC02D0DE6ADD6A0001000EAD5D86
:104C3000010EAE592DE2ADC000F0AEC001F0000E85
:104C4000D8800056010E015600C0E6FF01C0E6FF05
:104C5000ADC0E9FFAEC0EAFFE906000EEA5A000E59
:104C6000E926010EEA22EF50E66E000EAD25026E37
:104C7000010EAE21036E02C0E6FFE66EF8EC54F0C2
:104C8000046E050EE15C02E2E16AE552E16E045059
:104C9000FCD90A0EF3CFDBFFDB5001E13FD70A0E50
:104CA000DBCF00F0016A00BE016800C0E6FF01C072
:104CB000E6FF4F0E026E9F0E036E046A02C0E6FF0F
:104CC000E66E04C0E6FF800EE66E000EE66E3BEC7C
:104CD00056F0056E070EE15C02E2E16AE552E16E14
:104CE0000550800EE66E000EE66E87EC54F0E5523D
:104CF000E552010E366E040E0F011411146F36507A
:104D0000006E016A00C0F3FF01C0F4FF55D0D95016
:104D1000060FE96E000EDA20EA6EEECFE6FFEECF68
:104D2000E6FFEECFE6FFEFCFE6FF330E006E9F0EFD
:104D3000016E026A00C0E6FFE66E02C0E6FF800E6A
:104D4000E66E000EE66E3BEC56F0036E090EE15C7B
:104D500002E2E16AE552E16E0350800EE66E000E5B
:104D6000E66E87EC54F0E552E55282A402D0010EC3
:104D7000366E8090A70E006EA10E016E026A00C012
:104D8000E6FFE66E02C0E6FF800EE66E000EE66EFF
:104D90003BEC56F0036E050EE15C02E2E16AE5527F
:104DA000E16E0350800EE66E000EE66E87EC54F066
:104DB000E552E552F36AF46A0F0EE15C02E2E16A41
:104DC000E552E16EE552E5CFDAFFE7CFD9FF1200F9
:104DD0002A0E006E9F0E016E026A00C0E6FFE66EAC
:104DE00002C0E6FF800EE66E000EE66E3BEC56F06B
:104DF000036E050EE15C02E2E16AE552E16E0350EA
:104E0000800EE66E000EE66E87EC54F0E552E55239
:104E1000E66A010EE66EE66A000EE66E020EE66EC9
:104E2000F8EC54F0006E050EE15C02E2E16AE55236
:104E3000E16E005036C000F2010EE66EE66A1AEC32
:104E400051F0E552E552366A12001C0E006E9F0EBC
:104E5000016E026A00C0E6FFE66E02C0E6FF800E49
:104E6000E66E000EE66E3BEC56F0036E050EE15C5E
:104E700002E2E16AE552E16E0350800EE66E000E3A
:104E8000E66E87EC54F0E552E5520F01086B096BB2
:104E90000A6B0B6B146B106B116B126B136B8090A6
:104EA000A70E006EA10E016E026A00C0E6FFE66E5C
:104EB00002C0E6FF800EE66E000EE66E3BEC56F09A
:104EC000036E050EE15C02E2E16AE552E16E035019
:104ED000800EE66E000EE66E87EC54F0E552E55269
:104EE000366A1200D9CFE6FFDACFE6FFE1CFD9FF6D
:104EF000E2CFDAFFE652E652E652E652E6520F0100
:104F0000092B000E0A230B2308CFDFFF010E09CF68
:104F1000DBFF020E0ACFDBFF030E0BCFDBFF090E18
:104F2000006E9F0E016E026A00C0E6FFE66E02C0D0
:104F3000E6FF800EE66E000EE66E3BEC56F0036E6A
:104F4000050EE15C02E2E16AE552E16E0350800E7B
:104F5000E66E000EE66E87EC54F0E552E552D9CFCE
:104F6000E9FFDACFEAFFEECFE6FFEECFE6FFEECFC6
:104F7000E6FFEFCFE6FFD9CFE9FFDACFEAFFEECFCA
:104F8000E6FFEECFE6FFEECFE6FFEFCFE6FFF20E55
:104F9000006E9E0E016E026A00C0E6FFE66E02C061
:104FA000E6FF800EE66E000EE66E3BEC56F0036EFA
:104FB0000D0EE15C02E2E16AE552E16E0350800E03
:104FC000E66E000EE66E87EC54F0E552E552D9CF5E
:104FD000E9FFDACFEAFFEECFE6FFEECFE6FFEECF56
:104FE000E6FFEFCFE6FF1DEC16F0E552E552E55285
:104FF000E552E76E040EE7CFDBFFDB5039E0040E2D
:10500000DBCF00F0016A00BE016800C0E6FF01C00E
:10501000E6FFD9CFE9FFDACFEAFFEECFE6FFEECF2A
:10502000E6FFEECFE6FFEFCFE6FF0B0E026EA00E1F
:10503000036E046A02C0E6FFE66E04C0E6FF800E5F
:10504000E66E000EE66E3BEC56F0056E0B0EE15C74
:1050500002E2E16AE552E16E0550800EE66E000E56
:10506000E66E87EC54F0E552E552010E366E01D043
:10507000366A050EE15C02E2E16AE552E16EE55254
:10508000E5CFDAFFE7CFD9FF1200D9CFE6FFDACFBD
:10509000E6FFE1CFD9FFE2CFDAFF130EE12402E30E
:1050A000E168E652E16E08CF3DF009CF3EF00ACF4D
:1050B0003FF00BCF40F0426A010E436E446A456AEE
:1050C00087EC57F00A0E3DC0DBFF0B0E3EC0DBFF46
:1050D0000C0E3FC0DBFF0D0E40C0DBFF110EDB6A84
:1050E000120EDB6AD9500A0FE96E000EDA20EA6E62
:1050F000EECFE6FFEECFE6FFEECFE6FFEFCFE6FF27
:1051000008CFE6FF09CFE6FF0ACFE6FF0BCFE6FFA9
:1051100008CFE6FF09CFE6FF0ACFE6FF0BCFE6FF99
:10512000D90E006E9E0E016E026A00C0E6FFE66EAA
:1051300002C0E6FF800EE66E000EE66E3BEC56F017
:10514000036E110EE15C02E2E16AE552E16E03508A
:10515000800EE66E000EE66E87EC54F0E552E552E6
:10516000E66A010EE66E000EE66E010EE66E61EC7A
:105170003DF0E552E552E552E5521BEC21F0040EFC
:10518000F3CFDBFF050EF4CFDBFFD950040FE96E40
:10519000000EDA20EA6EEE50ED1005E0040EDBCFD3
:1051A00000F0050E07D30A0EDBCF00F00B0E0C0E3D
:1051B0000D0E010E0016016A026A036A005001100A
:1051C0000210031001E0FFD00A0EDBCF00F00B0E3F
:1051D000DBCF01F00C0EDBCF02F00D0EDBCF03F0C6
:1051E000D8900332023201320032090ED8900036D4
:1051F000013602360336E806F9E1012A000E0222E2
:105200000322060E00C0DBFF070E01C0DBFF080E05
:1052100002C0DBFF090E03C0DBFFD950060FE96EA9
:10522000000EDA20EA6EEECFE6FFEECFE6FFEECF1D
:10523000E6FFEFCFE6FF1DEC16F0E552E552E55232
:10524000E552E76E100EE7CFDBFFDB5007E0100EF4
:10525000DBCF00F0016A00AEAFD29BD2D9500E0F67
:10526000E66E000EDA20E66EE66A010EE66E000ECD
:10527000E66E030EE66E35EC10F0006E060EE15C95
:1052800002E2E16AE552E16E0050E76E100EE7CFF0
:10529000DBFFDB5007E0100EDBCF00F0016A00AE51
:1052A0008BD277D2100EDBCF00F0016A00BE01680E
:1052B00000C0E6FF01C0E6FFD950060FE96E000E00
:1052C000DA20EA6EEECFE6FFEECFE6FFEECFE6FFA6
:1052D000EFCFE6FF010E026E036A046A056AD95039
:1052E0000A0FE96E000EDA20EA6EEE500226EE504A
:1052F0000322EE500422EE50052202C0E6FF03C056
:10530000E6FF04C0E6FF05C0E6FFB80E066E9E0E7F
:10531000076E086A06C0E6FFE66E08C0E6FF800E6C
:10532000E66E000EE66E3BEC56F0096E0F0EE15C89
:1053300002E2E16AE552E16E0950800EE66E000E6F
:10534000E66E87EC54F0E552E552060EDBCF00F036
:10535000070EDBCF01F0080EDBCF02F0090EDBCF2A
:1053600003F00106000E025A035A060E00C0DBFFCE
:10537000070E01C0DBFF080E02C0DBFF090E03C0F1
:10538000DBFFD950060FE96E000EDA20EA6EEECF91
:10539000E6FFEECFE6FFEECFE6FFEFCFE6FF1DEC38
:1053A00016F0E552E552E552E552E76E100EE7CFF2
:1053B000DBFFDB5001E109D1100EDBCF00F0016A09
:1053C00000AEFAD1E6D10A0EDBCF3DF00B0EDBCFFB
:1053D0003EF00C0EDBCF3FF00D0EDBCF40F0D8904F
:1053E00040323F323E323D32426A020E436E446AE0
:1053F000456A22EC57F0060E39C0DBFF070E3AC0B3
:10540000DBFF080E3BC0DBFF090E3CC0DBFFD950C1
:10541000060FE96E000EDA20EA6EEECFE6FFEECF61
:10542000E6FFEECFE6FFEFCFE6FF1DEC16F0E5520C
:10543000E552E552E552E76E100EE7CFDBFFDB5099
:1054400007E0100EDBCF00F0016A00AEB5D1A1D1AC
:10545000D9500E0FE66E000EDA20E66EE66A010EF7
:10546000E66E000EE66E030EE66E35EC10F0006E92
:10547000060EE15C02E2E16AE552E16E0050E76E81
:10548000100EE7CFDBFFDBCF00F0016A00BE016842
:1054900000C0E6FF01C0E6FFD950060FE96E000E1E
:1054A000DA20EA6EEECFE6FFEECFE6FFEECFE6FFC4
:1054B000EFCFE6FF0A0EDBCF02F00B0EDBCF03F0DF
:1054C0000C0EDBCF04F00D0EDBCF05F00206000E54
:1054D000035A045A055A02C0E6FF03C0E6FF04C09F
:1054E000E6FF05C0E6FF960E066E9E0E076E086A82
:1054F00006C0E6FFE66E08C0E6FF800EE66E000E10
:10550000E66E3BEC56F0096E0F0EE15C02E2E16ADA
:10551000E552E16E0950800EE66E000EE66E87ECF5
:1055200054F0E552E552100EDB5007E0100EDBCFD1
:1055300000F0016A00AE40D12CD1D950060FE96EBF
:10554000000EDA20EA6EEECFE6FFEECFE6FFEECFFA
:10555000E6FFEFCFE6FF1DEC16F0E552E552E5520F
:10556000E552E76E100EE7CFDBFFDB5007E0100ED1
:10557000DBCF00F0016A00AE1FD10BD182B41BD08B
:10558000D9500E0FE66E000EDA20E66EE66A010EC6
:10559000E66E000EE66E030EE66EFDEC12F0006E97
:1055A000060EE15C02E2E16AE552E16E0050E76E50
:1055B000100EE7CFDBFF100EDB5007E0100EDBCF45
:1055C00000F0016A00AEF8D0E4D082B41BD0D9500C
:1055D0000E0FE66E000EDA20E66EE66A010EE66E4B
:1055E000000EE66E010EE66EFDEC12F0006E060E89
:1055F000E15C02E2E16AE552E16E0050E76E100EF6
:10560000E7CFDBFF100EDB5038E0100EDBCF00F0F1
:10561000016A00BE016800C0E6FF01C0E6FF860E19
:10562000026E9E0E036E046A02C0E6FFE66E04C0C0
:10563000E6FF800EE66E000EE66E3BEC56F0056E61
:10564000070EE15C02E2E16AE552E16E0550800E70
:10565000E66E000EE66E87EC54F0E552E552010E60
:10566000F36E110EF3CFDBFF120EDB6A100EDBCFF1
:1056700000F0016A00AEA0D08CD00A0EDBCF00F0A3
:105680000B0E0C0E0D0E010E0016016A026A036A63
:10569000005001100210031027E182B41BD0D95032
:1056A0000E0FE66E000EDA20E66EE66A010EE66E7A
:1056B000000EE66E030EE66EFDEC12F0006E060EB6
:1056C000E15C02E2E16AE552E16E0050E76E100E25
:1056D000E7CFDBFF100EDB5007E0100EDBCF00F052
:1056E000016A00AE69D055D082B419D0D9500E0FDE
:1056F000E66E000EDA20E66E000EE66EE66AE66EF4
:10570000E66AFDEC12F0006E060EE15C02E2E16A70
:10571000E552E16E0050E76E100EE7CFDBFF100E92
:10572000DB5039E0100EDBCF00F0016A00BE0168EB
:1057300000C0E6FF01C0E6FF710E026E9E0E036E12
:10574000046A02C0E6FFE66E04C0E6FF800EE66E65
:10575000000EE66E3BEC56F0056E070EE15C02E2D1
:10576000E16AE552E16E0550800EE66E000EE66ECF
:1057700087EC54F0E552E552010EF36E110EF3CFB3
:10578000DBFF120EDB6A100EDBCF00F0016A00AE09
:1057900013D0016811D0D950110FE96E000EDA2034
:1057A000EA6EEE50ED1002E172EC27F0110EDBCF45
:1057B00000F0120EDBCF01F000C0F3FF01C0F4FFD8
:1057C000130EE15C02E2E16AE552E16EE552E5CFDB
:1057D000DAFFE7CFD9FF1200E66A010EE66EE66A4D
:1057E000000EE66E020EE66EF8EC54F0006E050E4A
:1057F000E15C02E2E16AE552E16E00500201010E55
:10580000006F020E1E101E6E010EE66EE66A1AECA6
:1058100051F0E552E552FD0E1E141E6E1200D9CF56
:10582000E6FFDACFE6FFE1CFD9FFE2CFDAFFE652BB
:10583000E652E6520F01020E116F076F04CF00F01F
:10584000016A026A036A000E006C011E0122021E38
:105850000222031E032205CF04F0056A066A076AC6
:10586000180ED8900436053606360736E806F9E1F4
:105870000450002605500122065002220750032240
:1058800006CF08F0096A0A6A0B6A100ED89008362B
:1058900009360A360B36E806F9E1085000260950A9
:1058A00001220A5002220B50032207CF3DF03E6A2C
:1058B0003F6A406A426A010E436E446A456A22ECBE
:1058C00057F0005039240F01086F01503A20096F3A
:1058D00002503B200A6F03503C200B6FDE6ADD6AEA
:1058E000DECF00F0DDCF01F0140E005C000E015899
:1058F00051E2E66ADECFE9FFDDCFEAFF010EE926DD
:10590000000EEA22AD0EE926040EEA22EF50E66E02
:10591000DECFE9FFDDCFEAFFAD0EE926040EEA2275
:10592000EF50E66EE8EC19F0E552E552E552020E52
:10593000F3CFDBFFDBCFE6FFE66A690E006E9E0E5B
:10594000016E026A00C0E6FFE66E02C0E6FF800E4E
:10595000E66E000EE66E3BEC56F0036E070EE15C61
:1059600002E2E16AE552E16E0350800EE66E000E3F
:10597000E66E87EC54F0E552E552DECF00F0DDCF65
:1059800001F0020E0026000E012200C0DEFF01C061
:10599000DDFFA6D7E552E552E552E552E5CFDAFF45
:0659A000E7CFD9FF120061
:0A59A600306A316A0401FB6BFC6BF0
:1059B000020EFD6F80901200D9CFE6FFDACFE6FF2E
:1059C000E1CFD9FFE2CFDAFFE652FB0EDB5001E078
:1059D000EADFDF6AFD0EDB507F0BE76EFD0EE7CFDF
:1059E000DBFF315021E0FD0EDBCFE6FFE66AFC0E67
:1059F000DBCFE6FFE66AFBC4E6FFFCC4E6FF5A0E17
:105A0000006E9E0E016E026A00C0E6FFE66E02C0E6
:105A1000E6FF800EE66E000EE66E3BEC56F0036E7F
:105A20000B0EE15C46E243D0305021E0FD0EDBCFAF
:105A3000E6FFE66AFC0EDBCFE6FFE66AFBC4E6FFA4
:105A4000FCC4E6FF4B0E006E9E0E016E026A00C0A3
:105A5000E6FFE66E02C0E6FF800EE66E000EE66E22
:105A60003BEC56F0036E0B0EE15C23E220D0FD0E02
:105A7000DBCFE6FFE66AFC0EDBCFE6FFE66AFBC49F
:105A8000E6FFFCC4E6FF3D0E006E9E0E016E026A4C
:105A900000C0E6FFE66E02C0E6FF800EE66E000E76
:105AA000E66E3BEC56F0036E0B0EE15C02E2E16A3F
:105AB000E552E16E0350800EE66E000EE66E87EC56
:105AC00054F0E552E552FC0EDB5001E177D0FD0EBB
:105AD000DB50040804E0FD0EDB50140804E1070E5F
:105AE000DF6E04012CD1FD0EDB503F0802E1316A6C
:105AF00017D0FD0EDB505F0802E1306A11D0400E76
:105B0000F36EFD0EDBCFF4FFF350F45C0DE3FD0EFE
:105B1000DB50540809E3FD0EDB50400805E0306A15
:105B20000401FB6BFC6B47D0FD0EDB5040081AE113
:105B3000010E306E0401FB6BFC6B370E006E9E0E87
:105B4000016E026A00C0E6FFE66E02C0E6FF800E4C
:105B5000E66E000EE66E3BEC56F0036E050EE15C61
:105B600020E21DD0FD0EDB50200828E1010E316E31
:105B70000401FB6BFC6B310E006E9E0E016E026A1F
:105B800000C0E6FFE66E02C0E6FF800EE66E000E85
:105B9000E66E3BEC56F0036E050EE15C02E2E16A54
:105BA000E552E16E0350800EE66E000EE66E87EC65
:105BB00054F0E552E552F36AF46AFAD0620E040139
:105BC000FB1902E11B0EFC1901E1EDD00F0EFB19D0
:105BD00002E1270EFC1901E1E6D0580EFB1902E1A3
:105BE0001B0EFC1901E1D7D0F70EFB1902E11A0ECA
:105BF000FC1901E1D4D0F60EFB1902E11A0EFC19D2
:105C000001E1C5D0F50EFB1902E11A0EFC1901E104
:105C1000BCD0A40EFB1902E11A0EFC1901E1B0D0B0
:105C20009E0EFB1902E11A0EFC1901E1A2D09D0E95
:105C3000FB1902E11A0EFC1901E196D09C0EFB192A
:105C400002E11A0EFC1901E18AD09B0EFB1902E158
:105C50001A0EFC1901E17ED0920EFB1902E11A0E18
:105C6000FC1901E175D0F40EFB1902E11A0EFC19C2
:105C700069E0C20EFB1902E11A0EFC195EE0900EFB
:105C8000FB1902E11A0EFC193EE0FB5101E08BD03A
:105C9000FC5101E088D0FD0EDB50600804E130507B
:105CA00002E0030E4BD0FD0EDB50600804E13150E2
:105CB00002E0050E43D0FD0EDB50680806E13150CE
:105CC00004E0900EFB6F1A0EFC6FFD0EDB506808AF
:105CD00004E1305002E0020E31D0FD0EDB506A08C4
:105CE00006E1315004E0F40EFB6F1A0EFC6FFD0E5E
:105CF000DB50700858E1305056E0040EDF6EFB6B4D
:105D0000FC6B808050D0FD0EDB50020804E1920E47
:105D1000FB6F1A0EFC6FFD0EDB50030804E0FD0E56
:105D2000DB50FF0804E18080DF6A809008D0FD0E20
:105D3000DB50160838E1A40E2BD0020EDF6EFB6B91
:105D4000FC6B31D0FD0EDB5005082DE1F50E20D0A7
:105D50009B0E1ED0FD0EDBCFF7F49C0E19D0FD0E6E
:105D6000DBCFF8F49D0E14D0FD0EDBCFF9F49E0EC0
:105D70000FD0FD0EDBCFFAF4FB6BFC6B010E03D0F2
:105D8000FB6BFC6B060EDF6E0ED0F70E01D0F70E2C
:105D9000FB6F1A0E07D0FB6BFC6B040EDF6E0F0E51
:105DA000FB6F270EFC6FDF50016AF36E01C0F4FF3A
:105DB000E552E552E5CFDAFFE7CFD9FF1200200E1A
:105DC000006E9E0E016E026A00C0E6FFE66E02C023
:105DD000E6FF800EE66E000EE66E3BEC56F0036EBC
:105DE000050EE15C02E2E16AE552E16E0350800ECD
:105DF000E66E000EE66E87EC54F0E552E552020EB8
:105E00001E101E6E0201006B82A403D0130E02113D
:105E1000026F016B0D0E026F036B82A402D0600E45
:105E2000036F040EE66EE66A1AEC51F0E552E55295
:105E3000FD0E1E141E6E80901200D9CFE6FFDACF41
:105E4000E6FFE1CFD9FFE2CFDAFFE652E652E652B3
:105E5000E652E652F8C400F0016A026A036A00AE34
:105E600003D0016802680368040ED890003601363A
:105E700002360336E806F9E102C003F001C002F081
:105E800000C001F0006AD8900036013602360336B1
:105E9000F9C404F0056A066A076A04AE02D0056810
:105EA000066806C007F005C006F004C005F0046AE5
:105EB000040ED8900436053606360736E806F9E1B2
:105EC00004500026055001220650022207500322EA
:105ED000FAC408F0096A0A6A0B6A08AE02D00968B7
:105EE0000A680AC00BF009C00AF008C009F0086A85
:105EF00008500026095001220A5002220B500322AA
:105F000000C0DFFF010E01C0DBFF020E02C0DBFF9D
:105F1000030E03C0DBFFF8C400F0016A026A036AE3
:105F200000AE03D0016802680368040ED890003602
:105F3000013602360336E806F9E1D890003601361C
:105F400002360336F9C404F0056A066A076A04AE2D
:105F500003D0056806680768040ED8900436053635
:105F600006360736E806F9E10450002605500122FE
:105F70000650022207500322FAC408F0096A0A6A8E
:105F80000B6A08AE03D009680A680B68085000263F
:105F9000095001220A5002220B50032200C0E6FFE2
:105FA00001C0E6FF02C0E6FF03C0E6FFFAC40CF042
:105FB0000D6A0CBE0D680CC0E6FF0DC0E6FFF9C40B
:105FC0000EF00F6A0EBE0F680EC0E6FF0FC0E6FFB0
:105FD000F8C410F0116A10BE116810C0E6FF11C0BD
:105FE000E6FFF7C412F0136A12BE136812C0E6FF90
:105FF00013C0E6FF010E146E9E0E156E166A14C0D5
:10600000E6FFE66E16C0E6FF800EE66E000EE66E58
:106010003BEC56F0176E110EE15C02E2E16AE552CC
:10602000E16E1750800EE66E000EE66E87EC54F0BF
:10603000E552E552D9CFE9FFDACFEAFFEECFE6FF2E
:10604000EECFE6FFEECFE6FFEFCFE6FFD9CFE9FFD9
:10605000DACFEAFFEECFE6FFEECFE6FFEECFE6FFC8
:10606000EFCFE6FFEA0E006E9D0E016E026A00C0E1
:10607000E6FFE66E02C0E6FF800EE66E000EE66EFC
:106080003BEC56F0036E0D0EE15C02E2E16AE55274
:10609000E16E0350800EE66E000EE66E87EC54F063
:1060A000E552E552D9CFE9FFDACFEAFFEECFE6FFBE
:1060B000EECFE6FFEECFE6FFEFCFE6FF1DEC16F0EA
:1060C000E552E552E552E552E76E040EE7CFDBFFFD
:1060D000DB5036E0040EDBCF00F0016A00BE016841
:1060E00000C0E6FF01C0E6FFD9CFE9FFDACFEAFF43
:1060F000EECFE6FFEECFE6FFEECFE6FFEFCFE6FF17
:10610000D20E026E9D0E036E046A02C0E6FFE66EBA
:1061100004C0E6FF800EE66E000EE66E3BEC56F025
:10612000056E0B0EE15C02E2E16AE552E16E05509C
:10613000800EE66E000EE66E87EC54F0E552E552F6
:106140000401FD6B8090050EE15C02E2E16AE5521C
:10615000E16EE552E5CFDAFFE7CFD9FF1200D9CFE4
:10616000E6FFDACFE6FFE1CFD9FFE2CFDAFF090E93
:10617000E12402E3E168E652E16EF8C400F0016A4E
:10618000026A036A00AE03D0016802680368040E65
:10619000D8900036013602360336E806F9E1D89089
:1061A0000036013602360336F9C404F0056A066A81
:1061B000076A04AE03D0056806680768040ED89025
:1061C0000436053606360736E806F9E1045000269F
:1061D000055001220650022207500322FAC408F09B
:1061E000096A0A6A0B6A08AE03D009680A680B6874
:1061F00008500026095001220A5002220B500322A7
:1062000000C0E6FF01C0E6FF02C0E6FF03C0E6FFF4
:10621000FAC40CF00D6A0CBE0D680CC0E6FF0DC090
:10622000E6FFF9C40EF00F6A0EBE0F680EC0E6FF5F
:106230000FC0E6FFF8C410F0116A10BE116810C05C
:10624000E6FF11C0E6FFAE0E126E9D0E136E146ACD
:1062500012C0E6FFE66E14C0E6FF800EE66E000E8A
:10626000E66E3BEC56F0156E0F0EE15C02E2E16A61
:10627000E552E16E1550800EE66E000EE66E87EC7C
:1062800054F0E552E552020EDB6A030EDB6A040E9F
:10629000DB6A050EDB6AD950070FE66E000EDA20C6
:1062A000E66EE66A010EE66E000EE66E020EE66E21
:1062B00035EC10F0006E060EE15C02E2E16AE55298
:1062C000E16E0050E76E060EE7CFDBFF070EDBCF77
:1062D000E6FF080EDBCFE6FF060EDBCF00F0016A1B
:1062E00000BE016800C0E6FF01C0E6FF8D0E026E31
:1062F0009D0E036E046A02C0E6FFE66E04C0E6FF70
:10630000800EE66E000EE66E3BEC56F0056E090E52
:10631000E15C02E2E16AE552E16E0550800EE66E54
:10632000000EE66E87EC54F0E552E552FD0E1E14A9
:106330001E6E070EDBCFE6FF080EDBCFE6FF1AEC82
:1063400051F0E552E552070EDBCF00F0080EDBCF2F
:1063500001F0026A036AD950020FE96E000EDA20DA
:10636000EA6EEE500026EE500122EE500222EE5070
:106370000322020E00C0DBFF030E01C0DBFF040E90
:1063800002C0DBFF050E03C0DBFFD950020FE96E30
:10639000000EDA20EA6EEECFE6FFEECFE6FFEECF9C
:1063A000E6FFEFCFE6FF7B0E006E9D0E016E026AE8
:1063B00000C0E6FFE66E02C0E6FF800EE66E000E4D
:1063C000E66E3BEC56F0036E090EE15C02E2E16A18
:1063D000E552E16E0350800EE66E000EE66E87EC2D
:1063E00054F0E552E5520401FD6B8090090EE15C2A
:1063F00002E2E16AE552E16EE552E5CFDAFFE7CF6E
:10640000D9FF1200D9CFE6FFDACFE6FFE1CFD9FFFF
:10641000E2CFDAFF150EE12402E3E168E652E16E15
:10642000F8C400F0016A026A036A00AE03D0016892
:1064300002680368040ED89000360136023603362F
:10644000E806F9E1D8900036013602360336F9C481
:1064500004F0056A066A076A04AE03D00568066898
:106460000768040ED8900436053606360736E80667
:10647000F9E104500026055001220650022207507F
:106480000322FAC408F0096A0A6A0B6A08AE03D04C
:1064900009680A680B6808500026095001220A5052
:1064A00002220B50032200C0E6FF01C0E6FF02C03B
:1064B000E6FF03C0E6FFFAC40CF00D6A0CBE0D68DF
:1064C0000CC0E6FF0DC0E6FFF9C40EF00F6A0EBE69
:1064D0000F680EC0E6FF0FC0E6FFF8C410F0116AA7
:1064E00010BE116810C0E6FF11C0E6FF580E126E14
:1064F0009D0E136E146A12C0E6FFE66E14C0E6FF2E
:10650000800EE66E000EE66E3BEC56F0156E0F0E3A
:10651000E15C02E2E16AE552E16E1550800EE66E42
:10652000000EE66E87EC54F0E552E552F8C400F038
:10653000016A026A036A00AE03D001680268036858
:10654000040ED8900036013602360336E806F9E12B
:10655000D8900036013602360336F9C404F0056AD5
:10656000066A076A04AE03D0056806680768040E69
:10657000D8900436053606360736E806F9E10450A9
:106580000026055001220650022207500322FAC4B9
:1065900008F0096A0A6A0B6A08AE03D009680A683B
:1065A0000B6808500026095001220A5002220B50A5
:1065B00003220E0E00C0DBFF0F0E01C0DBFF100E2A
:1065C00002C0DBFF110E03C0DBFF060EDB6A070E05
:1065D000DB6A080EDB6A090EDB6A010EDE6EDD6A1D
:1065E0000E0EDBCF00F00F0E100E110E010E001676
:1065F000016A026A036A005001100210031001E0F0
:10660000DFD00E0EDBCF00F00F0EDBCF01F0100E4F
:10661000DBCF02F0110EDBCF03F0D8900332023251
:1066200001320032090ED8900036013602360336A8
:10663000E806F9E1012A000E022203220A0E00C038
:10664000DBFF0B0E01C0DBFF0C0E02C0DBFF0D0EEB
:1066500003C0DBFFD9500A0FE96E000EDA20EA6EA4
:10666000EECFE6FFEECFE6FFEECFE6FFEFCFE6FFA1
:106670001DEC16F0E552E552E552E552E76E120EBA
:10668000E7CFDBFFD950130FE66E000EDA20E66E7F
:10669000E66A010EE66E000EE66E030EE66E35EC5F
:1066A00010F0006E060EE15C02E2E16AE552E16E76
:1066B0000050E76E120EE7CFDBFFDBCF00F0016A80
:1066C00000BE016800C0E6FF01C0E6FFD9500A0F16
:1066D000E96E000EDA20EA6EEECFE6FFEECFE6FFBF
:1066E000EECFE6FFEFCFE6FF010E026E036A046A0B
:1066F000056AD9500E0FE96E000EDA20EA6EEE50F0
:106700000226EE500322EE500422EE50052202C073
:10671000E6FF03C0E6FF04C0E6FF05C0E6FF390E52
:10672000066E9D0E076E086A06C0E6FFE66E08C09C
:10673000E6FF800EE66E000EE66E3BEC56F0096E4C
:106740000F0EE15C02E2E16AE552E16E0950800E53
:10675000E66E000EE66E87EC54F0E552E5520A0E46
:10676000DBCF00F00B0EDBCF01F00C0EDBCF02F025
:106770000D0EDBCF03F00106000E025A035A0A0E7B
:1067800000C0DBFF0B0E01C0DBFF0C0E02C0DBFF05
:106790000D0E03C0DBFFD9500A0FE96E000EDA20A0
:1067A000EA6EEECFE6FFEECFE6FFEECFE6FFEFCFED
:1067B000E6FF1DEC16F0E552E552E552E552D8D061
:1067C0000E0EDBCF3DF00F0EDBCF3EF0100EDBCF19
:1067D0003FF0110EDBCF40F0D89040323F323E32D6
:1067E0003D32426A020E436E446A456A22EC57F01B
:1067F0000A0E39C0DBFF0B0E3AC0DBFF0C0E3BC0AC
:10680000DBFF0D0E3CC0DBFFD9500A0FE96E000E16
:10681000DA20EA6EEECFE6FFEECFE6FFEECFE6FF40
:10682000EFCFE6FF1DEC16F0E552E552E552E552DA
:10683000E76E120EE7CFDBFFD950130FE66E000EA6
:10684000DA20E66EE66A010EE66E000EE66E030ED4
:10685000E66E35EC10F0006E060EE15C02E2E16AD5
:10686000E552E16E0050E76E120EE7CFDBFFDBCFA3
:1068700000F0016A00BE016800C0E6FF01C0E6FF4B
:10688000D9500A0FE96E000EDA20EA6EEECFE6FF6D
:10689000EECFE6FFEECFE6FFEFCFE6FF0E0EDBCF4B
:1068A00002F00F0EDBCF03F0100EDBCF04F0110E61
:1068B000DBCF05F00206000E035A045A055A02C047
:1068C000E6FF03C0E6FF04C0E6FF05C0E6FF190EC1
:1068D000066E9D0E076E086A06C0E6FFE66E08C0EB
:1068E000E6FF800EE66E000EE66E3BEC56F0096E9B
:1068F0000F0EE15C02E2E16AE552E16E0950800EA2
:10690000E66E000EE66E87EC54F0E552E552D95083
:106910000A0FE96E000EDA20EA6EEECFE6FFEECF48
:10692000E6FFEECFE6FFEFCFE6FF1DEC16F0E552F7
:10693000E552E552E552E76E120EE7CFDBFF82B477
:106940001BD0D950130FE66E000EDA20E66EE66A11
:10695000010EE66E000EE66E030EE66EFDEC12F022
:10696000006E060EE15C02E2E16AE552E16E005063
:10697000E76E120EE7CFDBFFD9CFE9FFDACFEAFFF0
:10698000EE50ED1001E131D20001AD6BAE6B4FEC7A
:1069900052F0120EF3CFDBFF040EDB6A050EDB6A4A
:1069A000040EDBCF00F0050EDBCF01F0D8900150D4
:1069B00004E6500E005C000E015801E36BD1040E9A
:1069C000DBCF02F0050EDBCF03F0040ED8900236C9
:1069D0000336E806FBE100010250AD5D0350AE59FD
:1069E00001E258D1160E006E9D0E016E026A00C0C3
:1069F000E6FFE66E02C0E6FF800EE66E000EE66E73
:106A00003BEC56F0036E050EE15C02E2E16AE552F2
:106A1000E16E0350800EE66E000EE66E87EC54F0D9
:106A2000E552E552020EDB6A030EDB6A020EDBCF93
:106A300000F0030EDBCF01F0D890015004E6100EF9
:106A4000005C000E01585BE2040EDBCF04F0050E83
:106A5000DBCF05F0040ED89004360536E806FBE1DE
:106A6000020EDB500424026E030EDB500520036E81
:106A700000010250AD5D0350AE5941E3040EDBCF7F
:106A800000F0050EDBCF01F0040ED8900036013681
:106A9000E806FBE1020EDB500024E96E030EDB503A
:106AA0000120EA6E000EE926010EEA22EF50E66EA2
:106AB000E66A100E026E9D0E036E046A02C0E6FFC7
:106AC000E66E04C0E6FF800EE66E000EE66E3BEC5E
:106AD00056F0056E070EE15C02E2E16AE552E16EF6
:106AE0000550800EE66E000EE66E87EC54F0E5521F
:106AF000E552020EDB2A030E99E3DB2A97D70C0E30
:106B0000006E9D0E016E026A00C0E6FFE66E02C0D6
:106B1000E6FF800EE66E000EE66E3BEC56F0036E6E
:106B2000050EE15C02E2E16AE552E16E0350800E7F
:106B3000E66E000EE66E87EC54F0E552E552020E6A
:106B4000DB6A030EDB6A020EDBCF00F0030EDBCF45
:106B500001F0D890015004E6100E005C000E0158C0
:106B600001E391D0040EDBCF04F0050EDBCF05F07E
:106B7000040ED89004360536E806FBE1020EDB5021
:106B80000424026E030EDB500520036E0001025048
:106B9000AD5D0350AE5901E276D0040EDBCF00F0BC
:106BA000050EDBCF01F0040ED89000360136E80662
:106BB000FBE1020EDB500024E96E030EDB500120E6
:106BC000EA6E000EE926010EEA22EF50200834E2B8
:106BD000040EDBCF00F0050EDBCF01F0040ED890E1
:106BE00000360136E806FBE1020EDB500024E96EB8
:106BF000030EDB500120EA6E000EE926010EEA22A8
:106C0000EF50E66EE66A090E026E9D0E036E046A90
:106C100002C0E6FFE66E04C0E6FF800EE66E000EE0
:106C2000E66E3BEC56F0056E070EE15C02E2E16AAF
:106C3000E552E16E055018D0070E006E9D0E016EF4
:106C4000026A00C0E6FFE66E02C0E6FF800EE66E56
:106C5000000EE66E3BEC56F0036E050EE15C02E2C0
:106C6000E16AE552E16E0350800EE66E000EE66EBC
:106C700087EC54F0E552E552020EDB2A030E01E2E6
:106C800062D7DB2A60D7040EDB2A050E01E288D624
:106C9000DB2A86D6050E006E9D0E016E026A00C0CC
:106CA000E6FFE66E02C0E6FF800EE66E000EE66EC0
:106CB0003BEC56F0036E050EE15C02E2E16AE55240
:106CC000E16E0350800EE66E000EE66E87EC54F027
:106CD000E552E552ADC000F0AEC001F0026A036AB1
:106CE000D950060FE96E000EDA20EA6EEE5000264B
:106CF000EE500122EE500222EE500322060E00C09A
:106D0000DBFF070E01C0DBFF080E02C0DBFF090E30
:106D100003C0DBFFD950060FE96E000EDA20EA6EE1
:106D2000000EEE5C010EEE58000EEE58000EEE580E
:106D300002E3DE6ADD6A120EDBCF00F0016A00BEFC
:106D40000168FE0E001804E1015002E1DE6ADD6A0E
:106D500082B41CD0D950130FE66E000EDA20E66E16
:106D6000ADC0E6FFAEC0E6FF000EE66E010EE66EB9
:106D7000FDEC12F0006E060EE15C02E2E16AE55203
:106D8000E16E0050E76E120EE7CFDBFF120EDB5014
:106D900001E1F2D5120EDBCF00F0016A00BE0168FE
:106DA00000C0E6FF01C0E6FFF50E026E9C0E036E0A
:106DB000046A02C0E6FFE66E04C0E6FF800EE66EDF
:106DC000000EE66E3BEC56F0056E070EE15C02E24B
:106DD000E16AE552E16E0550800EE66E000EE66E49
:106DE00087EC54F0E552E552C7D50E0EDBCF00F02C
:106DF0000F0E100E110E010E0016016A026A036AD0
:106E000000500110021003101DE182B436D0D95099
:106E1000130FE66E000EDA20E66EE66A010EE66EED
:106E2000000EE66E030EE66EFDEC12F0006E060E2E
:106E3000E15C02E2E16AE552E16E0050E76E120E9B
:106E4000E7CFDBFF82B419D0D950130FE66E000EE6
:106E5000DA20E66E000EE66EE66AE66EE66AFDECA5
:106E600012F0006E060EE15C02E2E16AE552E16EAC
:106E70000050E76E120EE7CFDBFF120EDB502AE068
:106E8000120EDBCF00F0016A00BE016800C0E6FF11
:106E900001C0E6FFE00E026E9C0E036E046A02C0A3
:106EA000E6FFE66E04C0E6FF800EE66E000EE66EBC
:106EB0003BEC56F0056E070EE15C02E2E16AE5523A
:106EC000E16E0550800EE66E000EE66E87EC54F023
:106ED000E552E552D950060FE96E000EDA20EA6E4F
:106EE000EECFE6FFEECFE6FFEECFE6FFEFCFE6FF19
:106EF000C60E006E9C0E016E026A00C0E6FFE66ED2
:106F000002C0E6FF800EE66E000EE66E3BEC56F029
:106F1000036E090EE15C02E2E16AE552E16E0350A4
:106F2000800EE66E000EE66E87EC54F0E552E552F8
:106F3000ADD80401FD6B8090150EE15C02E2E16AC0
:106F4000E552E16EE552E5CFDAFFE7CFD9FF120057
:106F5000BD0E006E9C0E016E026A00C0E6FFE66E7A
:106F600002C0E6FF800EE66E000EE66E3BEC56F0C9
:106F7000036E050EE15C02E2E16AE552E16E035048
:106F8000800EE66E000EE66E87EC54F0E552E55298
:106F9000E66A010EE66EE66A000EE66E020EE66E28
:106FA000F8EC54F0006E050EE15C02E2E16AE55295
:106FB000E16E0050FDC400F2010EE66EE66A1AECC6
:106FC00051F0E552E5520401FD6B1200B10E006E66
:106FD0009C0E016E026A00C0E6FFE66E02C0E6FF8C
:106FE000800EE66E000EE66E3BEC56F0036E050E6C
:106FF000E15C02E2E16AE552E16E0350800EE66E6A
:10700000000EE66E87EC54F0E552E552E66A010E9A
:10701000E66EE66A000EE66E020EE66EF8EC54F0DE
:10702000006E050EE15C02E2E16AE552E16E00509D
:107030000201006B80900401FD6B1200A60E006E31
:107040009C0E016E026A00C0E6FFE66E02C0E6FF1B
:10705000800EE66E000EE66E3BEC56F0036E050EFB
:10706000E15C02E2E16AE552E16E0350800EE66EF9
:10707000000EE66E87EC54F0E552E5520401FA6B1F
:10708000F96BF86B80900401FD6B1200D9CFE6FF1D
:10709000DACFE6FFE1CFD9FFE2CFDAFFE652E652E0
:1070A000E652E652E6520401FA2B0F0EE76EFA1989
:1070B000E8AE02D0FA3503D0E750D880FA550FE297
:1070C000FA6BF92B010EE76EF919E8AE02D0F9352B
:1070D00003D0E750D880F95502E2F96BF82BF8C4D9
:1070E00000F0016A026A036A00AE03D00168026818
:1070F0000368040ED8900036013602360336E806DF
:10710000F9E102C003F001C002F000C001F0006A22
:10711000D8900036013602360336F9C404F0056A09
:10712000066A076A04AE02D00568066806C007F062
:1071300005C006F004C005F0046A040ED8900436B9
:10714000053606360736E806F9E1045000260550F4
:1071500001220650022207500322FAC408F0096AED
:107160000A6A0B6A08AE02D009680A680AC00BF006
:1071700009C00AF008C009F0086A08500026095042
:1071800001220A5002220B50032200C0DFFF010E31
:1071900001C0DBFF020E02C0DBFF030E03C0DBFFFA
:1071A000FAC400F0016A00BE016800C0E6FF01C039
:1071B000E6FFF9C402F0036A02BE036802C0E6FFFC
:1071C00003C0E6FFF8C404F0056A04BE056804C005
:1071D000E6FF05C0E6FFF7C406F0076A06BE0768CB
:1071E00006C0E6FF07C0E6FF870E086E9C0E096E1C
:1071F0000A6A08C0E6FFE66E0AC0E6FF800EE66E89
:10720000000EE66E3BEC56F00B6E0D0EE15C02E2FA
:10721000E16AE552E16E0B50800EE66E000EE66EFE
:1072200087EC54F0E552E552D9CFE9FFDACFEAFF17
:10723000EECFE6FFEECFE6FFEECFE6FFEFCFE6FFC5
:10724000D9CFE9FFDACFEAFFEECFE6FFEECFE6FFD8
:10725000EECFE6FFEFCFE6FFEA0E006E9D0E016E69
:10726000026A00C0E6FFE66E02C0E6FF800EE66E30
:10727000000EE66E3BEC56F0036E0D0EE15C02E292
:10728000E16AE552E16E0350800EE66E000EE66E96
:1072900087EC54F0E552E552D9CFE9FFDACFEAFFA7
:1072A000EECFE6FFEECFE6FFEECFE6FFEFCFE6FF55
:1072B0001DEC16F0E552E552E552E552E76E040E7C
:1072C000E7CFDBFFDB5036E0040EDBCF00F0016AD6
:1072D00000BE016800C0E6FF01C0E6FFD9CFE9FFAC
:1072E000DACFEAFFEECFE6FFEECFE6FFEECFE6FF26
:1072F000EFCFE6FFD20E026E9D0E036E046A02C04F
:10730000E6FFE66E04C0E6FF800EE66E000EE66E57
:107310003BEC56F0056E0B0EE15C02E2E16AE552D1
:10732000E16E0550800EE66E000EE66E87EC54F0BE
:10733000E552E5520401FD6B050EE15C02E2E16AF3
:10734000E552E16EE552E5CFDAFFE7CFD9FF120053
:10735000D9CFE6FFDACFE6FFE1CFD9FFE2CFDAFF00
:107360000A0EE12402E3E168E652E16EDF6A010EF3
:10737000DB6A020EDB6A030EDB6A090EDB6A070EAC
:10738000966E0F01010E1F6F0F01206B9292929467
:107390008082810ED56EC70ED56EF29434EC54F017
:1073A000490E006E9C0E016E026A00C0E6FFE66E9A
:1073B00002C0E6FF800EE66E000EE66E3BEC56F075
:1073C000036E050EE15C02E2E16AE552E16E0350F4
:1073D000800EE66E000EE66E87EC54F0E552E55244
:1073E0002C0EE66E9C0EE66E350EE66E9C0EE66E7C
:1073F000410E006E9C0E016E026A00C0E6FFE66E52
:1074000002C0E6FF800EE66E000EE66E3BEC56F024
:10741000036E090EE15C02E2E16AE552E16E03509F
:10742000800EE66E000EE66E87EC54F0E552E552F3
:10743000010EE66EE66A1B0E006E9C0E016E026A7D
:1074400000C0E6FFE66E02C0E6FF800EE66E000EAC
:10745000E66E3BEC56F0036E070EE15C02E2E16A79
:10746000E552E16E0350800EE66E000EE66E87EC8C
:1074700054F0E552E552FC50E66EE66A0E0E006EE0
:107480009C0E016E026A00C0E6FFE66E02C0E6FFD7
:10749000800EE66E000EE66E3BEC56F0036E070EB5
:1074A000E15C02E2E16AE552E16E0350800EE66EB5
:1074B000000EE66E87EC54F0E552E5528450E66E1D
:1074C000E66A020E006E9C0E016E026A00C0E6FFC4
:1074D000E66E02C0E6FF800EE66E000EE66E3BEC46
:1074E00056F0036E070EE15C02E2E16AE552E16EDE
:1074F0000350800EE66E000EE66E87EC54F0E55207
:10750000E552070E8414E76E090EE7CFDBFF00019A
:10751000A86BA96BAA6BAB6B2DEC56F0F20E006E4C
:107520009B0E016E026A00C0E6FFE66E02C0E6FF37
:10753000800EE66E000EE66E3BEC56F0036E050E16
:10754000E15C02E2E16AE552E16E0350800EE66E14
:10755000000EE66E87EC54F0E552E552F40EE66E4E
:10756000010EE66ED0EC55F0E552E552808469ECF0
:107570003FF0F3CFDBF0F3CF00F0016A00BE01680B
:1075800000C0E6FF01C0E6FFDA0E026E9B0E036E3E
:10759000046A02C0E6FFE66E04C0E6FF800EE66EF7
:1075A000000EE66E3BEC56F0056E070EE15C02E263
:1075B000E16AE552E16E0550800EE66E000EE66E61
:1075C00087EC54F0E552E5520001DB510EE0DBC0E0
:1075D00000F0016A00BE016800C0E6FF01C0E6FFDE
:1075E00081EC42F0E552E552FFD7F6EC3FF00001A6
:1075F000FB511CE0090EDBCFE6FFE66ACB0E006E06
:107600009B0E016E026A00C0E6FFE66E02C0E6FF56
:10761000E10EE66E000EE66E3BEC56F0036E070ED2
:10762000E15C02E2E16AE552E16E03500F011F5195
:107630001EE0BB0E006E9B0E016E026A00C0E6FFEC
:10764000E66E02C0E6FF800EE66E000EE66E3BECD4
:1076500056F0036E050EE15C02E2E16AE552E16E6E
:1076600003500001020EAF6F0001210E1DD0AB0EC2
:10767000006E9B0E016E026A00C0E6FFE66E02C05D
:10768000E6FF800EE66E000EE66E3BEC56F0036EF3
:10769000050EE15C02E2E16AE552E16E0350000191
:1076A000010EAF6F0001040EB06F800EE66E000E8B
:1076B000E66E87EC54F0E552E552080EDB6AE3EC27
:1076C00050F0E10EE66E000EE66E1DEC0FF0E55296
:1076D000E5520001DC6FE850DB6FDC51E66EE66AD4
:1076E000E10EE66E000EE66E960E006E9B0E016ECB
:1076F000026A00C0E6FFE66E02C0E6FF800EE66E9C
:10770000000EE66E3BEC56F0036E090EE15C02E201
:10771000E16AE552E16E0350800EE66E000EE66E01
:1077200087EC54F0E552E5520001DB513CE0DBC050
:1077300000F0016A00BE016800C0E6FF01C0E6FF7C
:1077400081EC42F0E552E5520001FB0528E1070E0D
:107750008414006E090EDB50005C21E0070E8414D7
:10776000E76E090EE7CFDBFFDBCFE6FFE66ACB0E65
:10777000006E9B0E016E026A00C0E6FFE66E02C05C
:10778000E6FFE10EE66E000EE66E3BEC56F0036E91
:10779000070EE15C02E2E16AE552E16E035099DB1B
:1077A000F3CFDBF08ED782A420D07C0E006E9B0E30
:1077B000016E026A00C0E6FFE66E02C0E6FF800EC0
:1077C000E66E000EE66E3BEC56F0036E050EE15CD5
:1077D00002E2E16AE552E16E0350800EE66E000EB1
:1077E000E66E87EC54F0E552E552D3EC2CF037EC22
:1077F00019F0060EDB6A070EDB6A8250020B01E00D
:1078000010D1D950060FE96E000EDA20EA6E050E8F
:10781000EE1801E1ED5001E104D10001FB0531E179
:10782000070E8414006E090EDB50005C2AE0070E80
:107830008414E76E090EE7CFDBFFDBCFE6FFE66AD5
:10784000CB0E006E9B0E016E026A00C0E6FFE66E74
:1078500002C0E6FFE10EE66E000EE66E3BEC56F06F
:10786000036E070EE15C02E2E16AE552E16E03504D
:10787000E10EE66E000EE66E87EC54F0E552E5523E
:10788000D0D00001AD6BAE6B80744FEC52F0080E9F
:10789000F3CFDBFFDB5009E0080EDB50006E016A1E
:1078A000FF0E001809E1015007E10001000ED88029
:1078B000AD55000EAE5531E2080EDBCFE6FFE66AAD
:1078C0006A0E006E9B0E016E026A00C0E6FFE66E55
:1078D00002C0E6FF800EE66E000EE66E3BEC56F050
:1078E000036E070EE15C02E2E16AE552E16E0350CD
:1078F000800EE66E000EE66E87EC54F0E552E5521F
:10790000ADC0E6FFAEC0E6FF000EE66E010EE66E0D
:10791000D8D8E552E552E552E5520001DB6B0F0184
:107920001F512AE0080EDB50070802E125EC27F082
:10793000080EDB0402E1F2EC1FF0080EDB50020837
:1079400002E191EC20F0080EDB50030808E166EC40
:1079500022F0060EF3CFDBFF070EF4CFDBFF080E9D
:10796000DB50050832E12CEC25F0060EF3CFDBFFEF
:10797000070EF4CFDBFF29D0080EDB50070802E129
:107980001EEC38F0080EDB50020802E1DFEC2EF0AE
:10799000080EDB0402E11DEC2FF0080EDB5003089B
:1079A00002E1AFEC30F0080EDB50040802E1A8EC75
:1079B00037F0080EDB50050802E102EC32F0080E49
:1079C000DB50060802E1E6EC37F00001A85101E1C6
:1079D00014D7A851E66EE66AA80EE66E000EE66EB3
:1079E0005B0E006E9B0E016E026A00C0E6FFE66E43
:1079F00002C0E6FF800EE66E000EE66E3BEC56F02F
:107A0000036E090EE15C02E2E16AE552E16E0350A9
:107A1000800EE66E000EE66E87EC54F0E552E552FD
:107A2000ECD681BC1BD0470E006E9B0E016E026A25
:107A300000C0E6FFE66E02C0E6FF800EE66E000EB6
:107A4000E66E3BEC56F0036E050EE15C02E2E16A85
:107A5000E552E16E035081BC19D0FDD7350E006EA2
:107A60009B0E016E026A00C0E6FFE66E02C0E6FFF2
:107A7000800EE66E000EE66E3BEC56F0036E050ED1
:107A8000E15C02E2E16AE552E16E0350800EE66ECF
:107A9000000EE66E87EC54F0E552E5528092E80E57
:107AA000E66E030EE66ED0EC55F0E552E5528082AC
:107AB000E80EE66E030EE66ED0EC55F0E552E552A8
:107AC00000D6D9CFE6FFDACFE6FFE1CFD9FFE2CF8C
:107AD000DAFFE652E652E652E652E652FA0EDBCF03
:107AE000E6FFFB0EDBCFE6FFFC0EDBCFE6FFFD0E75
:107AF000DBCFE6FF260E006E9B0E016E026A00C011
:107B0000E6FFE66E02C0E6FF800EE66E000EE66E51
:107B10003BEC56F0036E090EE15C02E2E16AE552CD
:107B2000E16E0350800EE66E000EE66E87EC54F0B8
:107B3000E552E552020EDB6A030EDB6A020EDBCF72
:107B400000F0030EDBCF01F0D890015004E6500E98
:107B5000005C000E015801E390D1020EDBCF02F071
:107B6000030EDBCF03F0040ED89002360336E8068E
:107B7000FBE1FA0EDBCF04F0FB0EDBCF05F0035088
:107B80000518E8AE02D0053404D00450025C05505C
:107B9000035801E372D1230E006E9B0E016E026A40
:107BA00000C0E6FFE66E02C0E6FF800EE66E000E45
:107BB000E66E3BEC56F0036E050EE15C02E2E16A14
:107BC000E552E16E0350800EE66E000EE66E87EC25
:107BD00054F0E552E552DE6ADD6ADECF00F0DDCF1B
:107BE00001F0D890015004E6100E005C000E015820
:107BF0006BE2020EDBCF04F0030EDBCF05F0040EC8
:107C0000D89004360536E806FBE1DE500424026E07
:107C1000DD500520036EFA0EDBCF06F0FB0EDBCF46
:107C200007F007500318E8AE02D0033404D0025026
:107C3000065C0350075848E3FC0EDBCF02F0FD0E54
:107C4000DBCF03F0DE500224006EDD500320016E16
:107C5000100E3F6E406A020EDBCF44F0030EDBCF06
:107C600045F05AEC57F000503D24E96E01503E209B
:107C7000EA6E040EEFCFDBFFDBCFE6FFE66A1D0EF8
:107C8000006E9B0E016E026A00C0E6FFE66E02C047
:107C9000E6FF800EE66E000EE66E3BEC56F0036EDD
:107CA000070EE15C02E2E16AE552E16E0350800EEC
:107CB000E66E000EE66E87EC54F0E552E552DF2AE0
:107CC000010E8BE3DB2A89D7190E006E9B0E016E25
:107CD000026A00C0E6FFE66E02C0E6FF800EE66EB6
:107CE000000EE66E3BEC56F0036E050EE15C02E220
:107CF000E16AE552E16E0350800EE66E000EE66E1C
:107D000087EC54F0E552E552DE6ADD6ADECF00F022
:107D1000DDCF01F0D890015004E6100E005C000E9B
:107D2000015801E3A3D0020EDBCF04F0030EDBCF3A
:107D300005F0040ED89004360536E806FBE1DE5067
:107D40000424026EDD500520036EFA0EDBCF06F030
:107D5000FB0EDBCF07F007500318E8AE02D0033468
:107D600004D00250065C0350075801E27FD0FC0E9D
:107D7000DBCF02F0FD0EDBCF03F0DE500224006EFD
:107D8000DD500320016E100E3F6E406A020EDBCF05
:107D900044F0030EDBCF45F05AEC57F000503D2481
:107DA000E96E01503E20EA6EEF50200839E2FC0EE9
:107DB000DBCF02F0FD0EDBCF03F0DE500224006EBD
:107DC000DD500320016E100E3F6E406A020EDBCFC5
:107DD00044F0030EDBCF45F05AEC57F000503D2441
:107DE000E96E01503E20EA6EEF50E66EE66A160E2E
:107DF000046E9B0E056E066A04C0E6FFE66E06C0C2
:107E0000E6FF800EE66E000EE66E3BEC56F0076E67
:107E1000070EE15C02E2E16AE552E16E075018D01C
:107E2000140E006E9B0E016E026A00C0E6FFE66E45
:107E300002C0E6FF800EE66E000EE66E3BEC56F0EA
:107E4000036E050EE15C02E2E16AE552E16E035069
:107E5000800EE66E000EE66E87EC54F0E552E552B9
:107E6000DF2A010E01E252D7DB2A50D7020EDB2AAD
:107E7000030E01E263D6DB2A61D6230E006E9B0E51
:107E8000016E026A00C0E6FFE66E02C0E6FF800EE9
:107E9000E66E000EE66E3BEC56F0036E050EE15CFE
:107EA00002E2E16AE552E16E0350800EE66E000EDA
:107EB000E66E87EC54F0E552E552050EE15C02E215
:107EC000E16AE552E16EE552E5CFDAFFE7CFD9FF8F
:107ED0001200D9CFE6FFDACFE6FFE1CFD9FFE2CF3C
:107EE000DAFFE652E652050EDE6EDD6A0001630E31
:107EF000DB6FDECF00F0DDCF01F0013466E2005031
:107F00000008000E015461E20001DB515EE0DF0673
:107F1000010E01E2DB06090E006E9B0E016E026A85
:107F200000C0E6FFE66E02C0E6FF800EE66E000EC1
:107F3000E66E3BEC56F0036E050EE15C02E2E16A90
:107F4000E552E16E0350800EE66E000EE66E87ECA1
:107F500054F0E552E552320EE66EE66AD0EC55F08A
:107F6000E552E552B10EE66E000EE66E11EC0AF037
:107F7000E552E5520001DB6F006E016A00BE016848
:107F800000C0E6FF01C0E6FFF60E026E9A0E036E19
:107F9000046A02C0E6FFE66E04C0E6FF800EE66EED
:107FA000000EE66E3BEC56F0056E070EE15C02E259
:107FB000E16AE552E16E0550800EE66E000EE66E57
:107FC00087EC54F0E552E55294D7DBC000F0016A2B
:107FD00000BE016800C0F3FF01C0F4FFE552E552A6
:107FE000E552E5CFDAFFE7CFD9FF1200D9CFE6FFA0
:107FF000DACFE6FFE1CFD9FFE2CFDAFF200EE124AE
:1080000002E3E168E652E16EE50E006E9A0E016E43
:10801000026A00C0E6FFE66E02C0E6FF800EE66E72
:10802000000EE66E3BEC56F0036E050EE15C02E2DC
:10803000E16AE552E16E0350800EE66E000EE66ED8
:1080400087EC54F0E552E552EF0EE66E000EE66E58
:108050001DEC0FF0E552E5520001DC6FE850DB6FDC
:10806000DC51E66EE66AEF0EE66E000EE66E960EE8
:10807000006E9B0E016E026A00C0E6FFE66E02C053
:10808000E6FF800EE66E000EE66E3BEC56F0036EE9
:10809000090EE15C02E2E16AE552E16E0350800EF6
:1080A000E66E000EE66E87EC54F0E552E5520001F4
:1080B000DB510AE0DBC000F0016A00BE016800C0CD
:1080C000F3FF01C0F4FF11D2D9500A0FE66E000E83
:1080D000DA20E66EE66A010EE66E000EE66E030E2C
:1080E000E66E35EC10F0006E060EE15C02E2E16A2D
:1080F000E552E16E00500001DB6F0A0EDBCFE6FFB8
:108100000B0EDBCFE6FFD50E006E9A0E016E026AF3
:1081100000C0E6FFE66E02C0E6FF800EE66E000ECF
:10812000E66E3BEC56F0036E070EE15C02E2E16A9C
:10813000E552E16E0350800EE66E000EE66E87ECAF
:1081400054F0E552E552020EDB6A030EDB6A040EC0
:10815000DB6A050EDB6A060EDB6A070EDB6A060EBB
:10816000DBCF00F0070EDBCF01F0D890015004E622
:108170000A0E005C000E015824E2D9500C0F006E6C
:10818000000EDA20016E060EDB500024E96E070EA9
:10819000DB500120EA6EEF6AD950160F006E000E18
:1081A000DA20016E060EDB500024E96E070EDB506C
:1081B0000120EA6EEF6A060EDB2A070ED0E3DB2A07
:1081C000CED7DE6ADD6ADECF00F0DDCF01F00A0E29
:1081D000DBCF02F00B0EDBCF03F00250005C03504C
:1081E000015801E358D1DECFE9FFDDCFEAFF000EF1
:1081F000E926030EEA22EF500D0801E0E0D0D95045
:10820000160FE66E000EDA20E66ED9500C0FE66E01
:10821000000EDA20E66EC90E006E9A0E016E026A3A
:1082200000C0E6FFE66E02C0E6FF800EE66E000EBE
:10823000E66E3BEC56F0036E090EE15C02E2E16A89
:10824000E552E16E0350800EE66E000EE66E87EC9E
:1082500054F0E552E552D9500C0FE66E000EDA20CC
:10826000E66EC30E006E9A0E016E026A00C0E6FF53
:10827000E66E02C0E6FF12EC55F0036E050EE15CFF
:1082800002E2E16AE552E16E035000090DE1D950C6
:10829000160FE66E000EDA20E66E5BEC55F0E55246
:1082A000E552F3500F011F6FD9500C0FE66E000E10
:1082B000DA20E66EBD0E006E9A0E016E026A00C0F4
:1082C000E6FFE66E02C0E6FF12EC55F0036E050E07
:1082D000E15C02E2E16AE552E16E035000090DE162
:1082E000D950160FE66E000EDA20E66E5BEC55F004
:1082F000E552E552F3500F01206FD9500C0FE66E96
:10830000000EDA20E66EB60E006E9A0E016E026A5C
:1083100000C0E6FFE66E02C0E6FF12EC55F0036E09
:10832000050EE15C02E2E16AE552E16E03500009EC
:108330000DE1D950160FE66E000EDA20E66E5BEC0A
:1083400055F0E552E552F3500001FB6F060EDB6A73
:10835000070EDB6A060EDBCF00F0070EDBCF01F065
:10836000D890015004E60A0E005C000E015824E289
:10837000D9500C0F006E000EDA20016E060EDB5095
:108380000024E96E070EDB500120EA6EEF6AD95037
:10839000160F006E000EDA20016E060EDB50002470
:1083A000E96E070EDB500120EA6EEF6A060EDB2A4B
:1083B000070ED0E3DB2ACED7040EDB6A1BD0DECF5C
:1083C000E9FFDDCFEAFF000EE926030EEA22EF50B7
:1083D0000A085BE0DECFE9FFDDCFEAFF000EE92609
:1083E000030EEA22EF5020080CE1010EF36E040E9A
:1083F000F3CFDBFF050EDB6A020EDB6A030EDB6ADE
:1084000044D0D950040FE96E000EDA20EA6EEE5027
:10841000ED100DE0DECFE9FFDDCFEAFF000EE9262B
:10842000030EEA22EF50E66ED950160F0CD0DECFC5
:10843000E9FFDDCFEAFF000EE926030EEA22EF5046
:10844000E66ED9500C0F006E000EDA20016E020E9F
:10845000DB500024E96E030EDB500120EA6EE5528A
:10846000E750EF6E020EDBCF00F0030EDBCF01F022
:10847000D890015004E60A0E005C000E015805E297
:10848000020EDB2A030E01E3DB2ADF2A010E01E2E2
:108490009AD6DB2A98D60F012051E66EE66A0F01C4
:1084A0001F51E66EE66AAA0E006E9A0E016E026A0F
:1084B00000C0E6FFE66E02C0E6FF800EE66E000E2C
:1084C000E66E3BEC56F0036E090EE15C02E2E16AF7
:1084D000E552E16E0350800EE66E000EE66E87EC0C
:1084E00054F0E552E552F36AF46A200EE15C02E2D0
:1084F000E16AE552E16EE552E5CFDAFFE7CFD9FF59
:108500001200D9CFE6FFDACFE6FFE1CFD9FFE2CF05
:10851000DAFF8092E80EE66E030EE66ED0EC55F0C0
:10852000E552E5528082E80EE66E030EE66ED0EC70
:1085300055F0E552E552FC0EDBCF00F0DB06FD0EF8
:10854000DBCF01F001E2DB06005001100EE080926B
:108550002C0EE66E010EE66ED0EC55F0E552E552BB
:1085600080822C0EE66E010EE1D78092F40EE66E4C
:10857000010EE66ED0EC55F0E552E5528082E552F0
:10858000E5CFDAFFE7CFD9FF1200D9CFE6FFDACF88
:10859000E6FFE1CFD9FFE2CFDAFFE652E652D6504E
:1085A000026E036AD750046E056A3F6A010E406E80
:1085B00004C044F005C045F05AEC57F002503D2489
:1085C000006E03503E2000C0DEFFDD6EF250040B53
:1085D00001E0010EE66EE66ADECFE6FFDDCFE6FFE4
:1085E0009A0E006E9A0E016E026A00C0E6FFE66EF9
:1085F00002C0E6FF800EE66E000EE66E3BEC56F023
:10860000036E090EE15C02E2E16AE552E16E03509D
:10861000800EE66E000EE66E87EC54F0E552E552F1
:10862000F294E552E552E552E5CFDAFFE7CFD9FF04
:02863000120036
:0E86320055EC48F0FB0EDBCFF3FFDB06F350F8
:1086400000090AE0A3EC48F0FA0E0EEC49F0F3E161
:10865000011CF1E1010E01D0000E84EF48F055EC51
:1086600048F03B0EE12402E3E168E652E16E010EC0
:10867000DB6A020EDB6AF90EDBCFF6FFFA0EDBCF08
:10868000F7FFFB0EDBCFF8FF0800F550DF6EDF5081
:1086900002E1A8EF47F0250EDF5C02E09BEF47F018
:1086A000030EDB6A040EDB6A050EDB6A060EDB6A6C
:1086B000070EDB6ABDEC47F02D0EDF5C0CE02B0EE5
:1086C000DF5C09E0200EDF5C06E0230EDF5C03E0E8
:1086D000300EDF5C1AE1DF50300A14E0130A0FE0BD
:1086E000030A0AE00B0A05E0060AE4E1030EDB8058
:1086F000E1D7030EDB82DED7030EDB84DBD7030E6C
:10870000DB86D8D7030EDB88D5D72A0EDF5C1BE1CA
:10871000B9EC47F007EC48F010E0030EDB803F684F
:108720004068130EDBCF44F0140EDBCF45F05AEC5B
:1087300057F0040E3DC0DBFF03D0130EF0EC47F002
:10874000BDEC47F00BD0090EDB6A5EEC48F003E0AD
:10875000D2EC48F0FAD7090EF0EC47F0030EDBB08C
:10876000DB982E0EDF5C1BE1BDEC47F02A0EDF5CD0
:108770000BE1B9EC47F007EC48F003E1130E42ECD3
:1087800048F0BDEC47F00BD0090EDB6A5EEC48F018
:1087900003E0D2EC48F0FAD7090E42EC48F0680E3C
:1087A000DF5C07E1BDEC47F0680EDF5C1DE1030E06
:1087B00018D0740EDF5C17E07A0EDF5C14E0480E10
:1087C000DF5C06E0540EDF5C03E05A0EDF5C02E182
:1087D000020E07D06C0EDF5C03E06A0EDF5C04E182
:1087E000010E95EC48F0C9DBDF506E0A01E17FD342
:1087F0001E0A01E192D1200A01E18FD13F0A01E175
:1088000049D11A0A01E146D10D0A01E143D1200AFA
:1088100001E140D13A0A01E13DD1200A01E13AD11A
:10882000260A01E135D10D0A01E132D11A0A01E12E
:10883000D9D0200A4AE0300A1FE0460A0EE0250A95
:1088400001E083D3D950F90FE96EFF0EDA20EA6E0A
:10885000010EEE5E000EEE5AEE5AA3EC48F0250E25
:10886000E66E95DB03E1011C01E169D39FEC48F062
:1088700001E26BD3DB2A69D3080EDB6A040EDB50FE
:10888000010806E2040EDB0467EC48F0DB508BDBEA
:10889000080EDB5009E0030EDB50010B05E172DB33
:1088A00001E04DD3080EDB6A64DBEFCFDFFF17EC8E
:1088B00049F003E1011C01E142D39FEC48F001E3E0
:1088C000DB2A60DB01E141D33AD3070EDB5002081B
:1088D0000FE1E3EC48F0030EAAEC48F00E0EEECFE9
:1088E000DBFF0F0EEECFDBFF100EEECFDBFF20D055
:1088F000F70EDBCF03F0F80EDBCF04F0020E035EC1
:10890000000E045AF70E03C0DBFFF80E04C0DBFFB5
:1089100003C0E9FF04C0EAFF9AEC48F0026A0E0EB9
:1089200000C0DBFF0F0E01C0DBFF100E02C0DBFF3B
:108930000E0EDBCFE6FF0F0EDBCFE6FF100EDBCF18
:10894000E6FF36EC55F0E552E552E552130E3EC017
:10895000DBFF140E3FC0DBFF060EDB5005E0130EFD
:10896000DEEC48F001E26ADB02EC49F002E2130EB1
:1089700037DBC5EC48F006E0040EDEEC48F002E21E
:10898000050E2EDB030EDBB005D0FCDA01E0D7D2FA
:10899000080EDB6A090EDB6A0E0EDBCFF6FF0F0E48
:1089A000DBCFF7FF100EDBCFF8FF0800F550DF6ECE
:1089B000DF5014E008EC49F011E217EC49F003E154
:1089C000011C01E1BCD2BBDB01E3DB2A090EDB2A7F
:1089D000D9500E0FE96E000ECBDBE7D7D3DA01E1F9
:1089E000B4D2ADD2C6DA110EEECFDBFF120EEDCF50
:1089F000DBFF110EDBCFE6FF120EDBCFE6FF28EC2C
:108A000055F0E552E552130EF3CFDBFF140EF4CF11
:108A1000DBFF060EDB5004E0130ED0DB01E20EDBC1
:108A200002EC49F002E2130EDBDAAFDB05E0040EE4
:108A3000C5DB02E2050ED4DA030EDBB005D0A2DA04
:108A400001E07DD2080EDB6A090EDB6A110EDBCF76
:108A5000E9FF120EDBCFEAFFEFCFDFFFDF5014E0BC
:108A6000D7DB12E2E4DB03E1011C01E168D267DB42
:108A700001E3DB2A090EDB2A110EDB2ADBCFE9FF3B
:108A8000120EE8E3DB2AE6D77DDA01E15ED257D2A7
:108A9000030EDB8E070EDB0410E195DB040E5ADBC0
:108AA0000A0EEECFDBFF0B0EEECFDBFF0C0EEECF90
:108AB000DBFF0D0EEECFDBFF6CD0070EDB500308A3
:108AC0002CE1030EDBAE0DD0B2DA020E76DAEFCF78
:108AD00000F0016A026A036A00AE39D001680268D8
:108AE00035D0F70EDBCF01F0F80EDBCF02F0020E2F
:108AF000015E000E025AF70E01C0DBFFF80E02C045
:108B0000DBFF01C0E9FF02C0EAFFEFCF00F00A0E71
:108B100000C0DBFF0B0EDB6A38D0070EDB5002080B
:108B200009E1030EDBAE04D059DB02AE10D00ED04B
:108B300055DB0DD0030EDBAE12D079DA020E3DDA32
:108B4000F9DA026A036A01AE02D002680368E2DA67
:108B50000C0E02C0DBFF0D0E03C0DBFF1AD0F70EB8
:108B6000DBCF02F0F80EDBCF03F0020E025E000E48
:108B7000035AF70E02C0DBFFF80E03C0DBFF02C092
:108B8000E9FF03C0EAFFD6DAC5DA0C0EDB6A0D0E88
:108B9000DB6A060EDB5005E1010EF36E050EF3CF26
:108BA000DBFF150EDB6A160EDB6AD950370F006E3D
:108BB000000EDA20016E390E00C0DBFF3A0E01C054
:108BC000DBFF380EDB6A080EDB6A0A0EAEDADF5016
:108BD000780A12E0200A10E0280A0CE0200A0AE0D5
:108BE0003F0A06E00D0A02E0200A08E1020E05D065
:108BF000080E03D0080EDF26100E97DA030EDBBE38
:108C000002D0DB92DB94DB50800B24E08ADAD89030
:108C1000030EEB50000A08E6000EEE5C000EEE5864
:108C2000000EEE58000EEE5815E213DA4268436863
:108C30004468456822EC57F00A0E39C0DBFF0B0E82
:108C40003AC0DBFF0C0E3BC0DBFF0D0E3CC0DBFF70
:108C50002D0E08D0030EDBA202D02B0E03D0DBA416
:108C600008D0200EF36E170EF3CFDBFF150EDB2AB4
:108C700002D0170EDB6A050EDB5003E1B7D901E124
:108C800089D0200E006EB00E016E000E026E070E2F
:108C9000DBCF03F0046A056A066A03C042F004C031
:108CA00043F005C044F006C045F0D3D987EC57F037
:108CB00000503924F36E01503A20F46E02503B20EC
:108CC000F86EF4CFF7FFF3CFF6FF0800090EF5CFEB
:108CD000DBFF580EDF5C0FE1610EF36E090E7BD9EE
:108CE0000AE3200E006E090EDBCFE7FF0050E75EBF
:108CF000090EE7CFDBFF070EDBCF00F0016A026A47
:108D0000036A0FDA00C042F001C043F002C044F031
:108D100003C045F0EECF3DF0EECF3EF0EECF3FF09A
:108D2000EFCF40F087EC57F040C0EDFF3FC0EDFFC4
:108D30003EC0EDFF3DC0EFFF390EDBCFE9FFDB06A4
:108D40003A0EDBCFEAFF01E2DB06090EDBCFEFFFD5
:108D5000150EDB2A4BD995E1030EDBA61DD06F0E55
:108D6000DF5C06E1C1D918E3150EDB285BDA14D00D
:108D7000780EDF5C09E0580EDF5C06E0620EDF5C17
:108D800003E0420EDF5C08E1020EF36E160EF3CF35
:108D9000DBFF02D0150EDB6A030EDB50100B0EE07A
:108DA000040EDBCF00F0050EDB50D880005406E245
:108DB000060EDB5003E1040EDB5034DA95D90AE2EB
:108DC000050EDBCFE7FF150EDB50E75E050EE7CFA4
:108DD000DBFF02D0050EDB6A040EDBCF00F0160EBF
:108DE00045D9D880005414E2160EDBCFE6FF150EED
:108DF000DBCFE6FF040EDBCFE6FF050EDB50E552CE
:108E0000E75CE552D880E754E552D880E7545FD953
:108E1000030EDB50010B0BE1080EDB5008E0B2D86B
:108E200001E08DD0080EDB50BED8080EDB6A170EAD
:108E3000DB5007E088D9170EF1D903E1011C01E1ED
:108E40007ED0160EDB5016E07ED9300EE66E9FD82F
:108E500002E1011C74E077D9DFCFE6FFE0EC56F0C9
:108E6000E552E552E552F4CF01F00001F31C02E1B6
:108E7000011C65E0050EDBCF00F0160EDB50D8803C
:108E8000005409E2050EDBCFE7FF160EDB50E75E6C
:108E9000050EE7CFDBFF300EE66E050ECBD94FE1B6
:108EA000390EDB2ADBCFE9FF3A0E01E3DB2ADBCF09
:108EB000EAFF090EEFCFDBFFDB500EE044D9090ECD
:108EC000ADD902E1011C3BE0390EDB2ADBCFE9FF23
:108ED0003A0EEDE3DB2AEBD755D831E1160EDBCFA6
:108EE000E6FF080EC3D8E552E7245DD82ED0070E62
:108EF000DB50030A1CE0010A14E0030A07E07BD9F7
:108F0000DBCFEEFF020EDBCFEDFF1FD0F5D8056AF9
:108F100003AE02D0046805682CD8BCD805C0EEFFAB
:108F200014D0EAD803BE046824D8B4D80ED063D9CC
:108F3000DBCFEFFF0AD07BD905E1011C03E1F36829
:108F4000F46810D0FCD801E3DB2A79D944EF43F070
:108F5000010EDBCF00F0020EDBCF01F000C0F3FF0B
:108F600001C0F4FF3B0EE15C02E2E16AE552E16E12
:108F7000CBD029D9020EAAEF48F061D90800F550EC
:108F8000DF6E1200200EE66E080E1AEF49F0E0ECDC
:108F900056F0E552E552E552F3CF00F0F4CF01F080
:108FA0000001F31C1200006E016AD950010F4DD967
:108FB0000050EE260150ED221200045E000E055A0C
:108FC000F70E04C0DBFFF80E05C0DBFF04C0E9FFAD
:108FD00005C0EAFF1200DBCFF4FFF350F45C12008F
:108FE000DB50E76E040EE7CFDBFF12000A0EDBCF8B
:108FF00000F00B0EDBCF01F00C0EDBCF02F00D0EFC
:10900000DBCF03F000500110021003101200130E0A
:10901000EECFDBFF140EEDCFDBFF130EDBCF00F046
:10902000140EDBCF01F00001800E01141200F70EC8
:10903000DBCF04F0F80EDBCF05F01200050EDB509D
:10904000E66ED950130F01D9E552E750EE6EED6A86
:1090500012000A0EDBCF3DF00B0EDBCF3EF00C0E04
:10906000DBCF3FF00D0EDBCF40F01200DBCFE6FF91
:10907000150EDBCFE6FF050EDB50E552E724E55287
:10908000E7241200DB50CED8010EF36E060EF3CFAC
:10909000DBFF1200EE50EFCFEAFFE96E02C0EEFFF9
:1090A00003C0EEFF04C0EEFF1200D9CFE6FFDACF17
:1090B000E6FFE1CFD9FFE2CFDAFF1200DFCFE6FF14
:1090C000E66AC2EC57F0E552E552F3501200E76E43
:1090D000080EE7CFDBFF1200EECF00F0EECF01F07D
:1090E000EFCF02F0036A1200050EDBCF00F0150E81
:1090F000DB50D88000541200010EDBCF02F0020ECC
:10910000DBCF03F0046A1200E552E5CFDAFFE7CFC8
:10911000D9FF12000A0E00C0DBFF0B0E01C0DBFFFF
:109120001200D9500A0F25EF49F0F36E070EF3CF66
:10913000DBFF1200EECF00F0EFCF01F01200010EC6
:10914000DB2A020E1200FC0EDBCFE6FFFD0EDBCFAA
:10915000E6FF1200005E000E015AF70E00C0DBFFB2
:10916000F80E01C0DBFF00C0E9FF01C0EAFF1200FA
:10917000DA20EA6EEF2AEECFF6FF000EEF22EECFF6
:10918000F7FFEF22EECFF8FF1200040EDBCFE6FF71
:10919000130EDB50E552E75C9ADFDB5004DF060E6E
:1091A000DB501200090EDB500A0DF350DF24D00F04
:1091B000E76E090EE7CFDBFFBDEF47F0DB50F36E44
:1091C000050EEBEF47F0F70EDBCF00F0F80EDBCF2C
:1091D00001F01200DFCFE6FFC7EF47F028DF030EF4
:1091E000ECDE6CEF48F019EC43F0E552E552E55245
:1091F000E55200091200BDDEEE50EFCFEAFFE96E46
:10920000010E1200130EDB50F36E040EEBEF47F06D
:10921000040EDB50F36E090EEBEF47F0DBCFE6FFF9
:10922000C7EF47F0E76E050EE7CFDBFF12008BDFDD
:10923000EAEF48F0DBCFE6FF86DFF3EF48F0D950E6
:10924000F90FE96EFF0EB8EF48F0E96E000EDA2074
:04925000EA6E1200B0
:0C925400D9CFE6FFDACFE6FFE1CFD9FF6B
:10926000E2CFDAFFFD0EDB5003E0C66A010E02D04A
:10927000C66A020EC66E400EC76EC68AE552E5CFBC
:10928000DAFFE7CFD9FF1200D9CFE6FFDACFE6FF4A
:10929000E1CFD9FFE2CFDAFFE652E652500EDE6EA2
:1092A000DD6AD9CFE9FFDACFEAFFEE06000EED5A0C
:1092B000EECF00F0EDCF01F000500110F2E1E552E9
:1092C000E552E552E5CFDAFFE7CFD9FF1200D9CF5B
:1092D000E6FFDACFE6FFE1CFD9FFE2CFDAFFFD0EFE
:1092E000DB50C96EC7B0FED7C7A0FED7FD0EC9CFF1
:1092F000DBFFE552E5CFDAFFE7CFD9FF1200C968FF
:10930000C7B0FED7C7A0FED7C9501200D9CFE6FF1D
:10931000DACFE6FFE1CFD9FFE2CFDAFFE652E6523D
:10932000FD0EDBAE18D0FD0EDB9EE66AE66AE66A4D
:10933000E66A770EE66EEADF006E050EE15C02E299
:10934000E16AE552E16E0050E76E010EE7CFDBFF08
:10935000DB50010874E38280D2DF8290D0DFFD0E03
:10936000DBCFE6FFB4DFE552F90EDBCF00F0FA0EFB
:10937000DBCF01F0FB0EDBCF02F0FC0EDBCF03F006
:10938000180ED8900332023201320032E806F9E1B9
:109390000050E66E9CDFE552F90EDBCF00F0FA0ECE
:1093A000DBCF01F0FB0EDBCF02F0FC0EDBCF03F0D6
:1093B000100ED8900332023201320032E806F9E191
:1093C0000050E66E84DFE552F90EDBCF00F0FA0EB6
:1093D000DBCF01F0FB0EDBCF02F0FC0EDBCF03F0A6
:1093E000080ED8900332023201320032E806F9E169
:1093F0000050E66E6CDFE552F90EDBCFE6FF67DF6B
:10940000E552010EDF6EFD0EDB50400802E1950EC5
:10941000DF6EFD0EDB50480802E1870EDF6EDFCF06
:10942000E6FF55DFE5520A0EDF6E69DFE76E010EDB
:10943000E7CFDBFFDB50800B02E0DF06F6E1010E39
:10944000DB50E552E552E552E5CFDAFFE7CFD9FF31
:109450001200D9CFE6FFDACFE6FFE1CFD9FFE2CFA6
:10946000DAFF090EE12402E3E168E652E16EE66A02
:10947000F1DEE552720ED36E0001FC5113E0825012
:10948000010B10E1E66AE66AE66AE66A000EE66E3D
:10949000E66A1BDA006E060EE15C02E2E16AE55262
:1094A000E16E005082800A0EDF6EDF5003E027DF9E
:1094B000DF06FBD7020EDB6AE66AE66AE66AE66A60
:1094C000400EE66E23DF006E050EE15C02E2E16A0B
:1094D000E552E16E0050010801E008D1AA0EE66EE7
:1094E000010EE66EE66AE66A480EE66E0FDF006E73
:1094F000050EE15C02E2E16AE552E16E005001080E
:1095000001E08DD0DF6A040EDF5C14E2F8DEE66E67
:10951000D950030F006E000EDA20016EDF500F01EC
:109520000024E96E000E0120EA6EE552E750EF6E6E
:10953000DF2AE9D7050EDB0401E0D8D0060EDB50A8
:10954000AA0801E0D3D0100EF36E070EF3CFDBFFB5
:10955000270EF36E080EF3CFDBFFD950070FE96E2D
:10956000000EDA20EA6EEE50ED1019E0E66AE66AC7
:10957000E66A400EE66EE90EE66EC8DE006E050E87
:10958000E15C02E2E16AE552E16E0050000907E0A9
:109590007BDE070EDB06080EE0E2DB06DED7D950E5
:1095A000070FE96E000EDA20EA6EEE50ED1001E1D1
:1095B0009DD0E66AE66AE66AE66A7A0EE66EA6DE9E
:1095C000006E050EE15C02E2E16AE552E16E0050D8
:1095D000000901E08BD0DF6A040EDF5C14E28FDE4D
:1095E000E66ED950030F006E000EDA20016EDF50D8
:1095F0000F010024E96E000E0120EA6EE552E750EB
:10960000EF6EDF2AE9D7030EDB50400B02E00C0EB1
:1096100001D0040EE76E020EE7CFDBFF67D0E66AEB
:10962000E66AE66AE66AE90EE66E70DE006E050E30
:10963000E15C02E2E16AE552E16E0050010805E3F7
:10964000020EDB6EDE52E90E07D0010EF36E020E43
:10965000F3CFDBFFDE52410EDD6E100EF36E070E10
:10966000F3CFDBFF270EF36E080EF3CFDBFFD950ED
:10967000070FE96E000EDA20EA6EEE50ED1019E0E9
:10968000E66AE66AE66AE66A010EDBCFE6FF3EDEE0
:10969000006E050EE15C02E2E16AE552E16E005007
:1096A000000907E0F1DD070EDB06080EE0E2DB064D
:1096B000DED7D950070FE96E000EDA20EA6EEE50C1
:1096C000ED1012E0E66A020EE66EE66AE66A500EF9
:1096D000E66E1CDE006E050EE15C02E2E16AE55218
:1096E000E16E0050000902E0020EDB6A020EDBCFE1
:1096F000FCF0828004DE010EE66EACDDE552D36A3A
:10970000020EDB5002E0000E01D0010E006E090EC9
:10971000E15C02E2E16AE552E16E0050E552E5CF1C
:10972000DAFFE7CFD9FF1200D9CFE6FFDACFE6FFA5
:10973000E1CFD9FFE2CFDAFFE652E652E652E65237
:109740000001FCB712D0D950F80FE96EFF0EDA20F5
:10975000EA6E090EE76ED890EF36010EEB36020E78
:10976000EB36030EEB36E706F6E1010EDF6ED9505D
:10977000F80FE96EFF0EDA20EA6EEECFE6FFEECFCD
:10978000E6FFEECFE6FFEFCFE6FF510EE66EBEDD61
:10979000006E050EE15C02E2E16AE552E16E005006
:1097A000000901E081D0400EF36E020EF3CFDBFF23
:1097B0009C0EF36E030EF3CFDBFFA1DDE76E010E0F
:1097C000E7CFDBFFDB50FF080CE1020EDB06DBCF4F
:1097D00000F0030E01E2DB06DBCF01F000500110C8
:1097E000ECE1010EDB50FE085FE1F60EDBCF02F08C
:1097F000F70EDBCF03F0020ED88002560356F40EAC
:10980000DB50025C006EF50EDB500358016E020E59
:1098100000C0DBFF030E01C0DBFFD950F60FE96E7D
:10982000FF0EDA20EA6EEE50ED100DE068DDF60E68
:10983000DB06DBCF00F0F70E01E2DB06DBCF01F049
:1098400000500110F3E1D950FC0FE96EFF0EDA2051
:10985000EA6EEE50ED101AE052DDE66EFC0EDBCF44
:10986000E9FFDB2AFD0EDBCFEAFF01E3DB2AE5524D
:10987000E750EF6EF40EDB06DBCF00F0F50E01E2F1
:10988000DB06DBCF01F000500110E6E138DD020E0F
:10989000DB06DBCF00F0030E01E2DB06DBCF01F0DD
:1098A00000500110F3E1DF6A828029DDDF50006E95
:1098B000040EE15C02E2E16AE552E16E0050E5521D
:1098C000E5CFDAFFE7CFD9FF1200D9CFE6FFDACF35
:1098D000E6FFE1CFD9FFE2CFDAFFE652E652E652E9
:1098E000010EDF6ED950FC0FE96EFF0EDA20EA6E32
:1098F000EE50ED1030E0F80EDBCF3FF0F90EDBCF8D
:1099000040F0DE523FC0DEFF40C0DDFFDD52D950E7
:10991000010FE96E000EDA20EA6EEE50ED1067E0FE
:109920000001FD51FE1163E0FC0EDBCFE9FFDB2AF5
:10993000FD0EDBCFEAFF01E3DB2AEF50E66EC7DC6A
:10994000E5520001FD07000EFE5B010EDB06020E74
:10995000DEE2DB06DCD7F80EDBCF00F0F90EDBCF62
:1099600001F0FA0EDBCF02F0FB0EDBCF03F000506C
:109970000110021003103DE00001FCB712D0D950D5
:10998000F80FE96EFF0EDA20EA6E090EE76ED89046
:10999000EF36010EEB36020EEB36030EEB36E70622
:1099A000F6E1D950F80FE96EFF0EDA20EA6EEECF3D
:1099B000E6FFEECFE6FFEECFE6FFEFCFE6FF580E75
:1099C000E66EA4DC006E050EE15C02E2E16AE5529F
:1099D000E16E0050000957E1E66879DCE552FE0EC1
:1099E000E66E75DCE5520001FD6B020EFE6FDF6A6C
:1099F0004AD0020E0001016AFD25006EFE510122CF
:109A0000010E00C0DBFF020E01C0DBFF010EDBCF49
:109A100000F0DB06020EDBCF01F001E2DB060050B6
:109A2000011004E0E66A53DCE552F0D768DC1F0B56
:109A3000050827E1880EF36E010EF3CFDBFF130E4E
:109A4000F36E020EF3CFDBFF5ADCFF0810E0D950B3
:109A5000010FE96E000EDA20EA6EEE50ED1007E01D
:109A600013DC010EDB06020EEFE2DB06EDD7D95068
:109A7000010FE96E000EDA20EA6EEE50ED1001E003
:109A8000DF6A82803CDCDF50E552E552E552E55268
:0A9A9000E5CFDAFFE7CFD9FF12009F
:069A9A000D0A5469636B24
:109AA000733A25752025640D0A000D0A503A256485
:109AB00020443A25640044534B53454C00444542EE
:109AC00055470050524F544F000D0A4B3A25732012
:109AD000563A2573000D0A526561642025642062A0
:109AE00079746573000D0A52656164696E6720635D
:109AF0006F6E666967000D0A4D6F756E7420726532
:109B00007475726E73202558000D0A4D6F756E7452
:109B1000696E67002E00256300207C200020253020
:109B20003258000D0A000D0A44756D70202558202A
:109B300025580D0A000D0A0D0A4F6F70732E204E26
:109B40006F2063617264000D0A0D0A496E746572BC
:109B50006661636520636C656172000D0A45646728
:109B6000653A2025732020256400202D2053746140
:109B70007475733A20256420200D0A000D0A436194
:109B800072642069732077726974652070726F74D3
:109B90006563746564000D0A4F70656E202573203F
:109BA00072657475726E73202558000D0A416D69D7
:109BB000676F2039313231440D0A000D0A53532F9B
:109BC000383020393133344C0D0A002F6C6966640B
:109BD00061746125642E62696E000D0A0D0A53449A
:109BE0005F6D6F756E742072657475726E7320256B
:109BF00064000D0A48617264776172652050500DEF
:109C00000A000D0A504F5254453A202558000D0ABB
:109C100053544B5054523A202558000D0A534420B7
:109C2000535049204449563A2025640031393A318D
:109C3000373A3130004D61722032342032303138C1
:109C4000000D0A2553202553000D0A0D0A485044E3
:109C500069736B207620302E3233000D0A25643A6A
:109C60002575202564007B4552527D002553007BDD
:109C7000505025647D000D0A5458434D44206C65B6
:109C80006E3A20256420000D0A414D3A20496E634A
:109C900072656D656E743A20256420256420256404
:109CA0002025642C20000D0A414D3A436C656172F9
:109CB000000D0A414D3A57616B657570000D0A4100
:109CC0004D3A44534A000D0A414D3A4275666620AA
:109CD000777220256C642062797465732072780035
:109CE0000D0A436C6F73696E672077722066616935
:109CF0006C202564000D0A577269746520666169DD
:109D00006C202564000A002E00256300207C2000C2
:109D10002025303258000D0A000D0A526420657665
:109D2000656E20736563746F723A20256C642061E0
:109D30007420256C58202564000D0A5264206F643D
:109D40006420736563746F723A20256C64206174BB
:109D500020256C58202564000D0A414D3A42756655
:109D60006620777220632F682F733A2025642F2591
:109D7000642F256420733A256C64000D0A20256C3D
:109D8000642062797465732073656E74000D0A52E5
:109D90006561642072657475726E732025582C207D
:109DA00025642062797465732072656164000D0A10
:109DB000414D3A4275666620726420632F682F73A6
:109DC0003A2025642F25642F256420733A256C647E
:109DD00020000D0A5365656B20746F20256C64208C
:109DE0006661696C6564202564000D0A5365656BC6
:109DF000696E6720746F20256C642028256C5829B3
:109E0000000D0A414D3A205365656B3A20256420C8
:109E100025642025642025642C20733A256C640079
:109E20000D0A414D3A53656E642073746174757305
:109E3000005B4D4C415D005B4D54415D007B2575E1
:109E40002025647D5B253032585D007B54257520CC
:109E500025647D5B253032585D007B4C25752025BF
:109E6000647D5B253032585D000D0A72633D2564C8
:109E7000000D0A436C6F73696E672077722066610C
:109E8000696C202564000D0A57726974652066614B
:109E9000696C202564000D0A5264206576656E2089
:109EA000736563746F723A20256C64206174202599
:109EB0006C582025640D0A000D0A5264206F6464FA
:109EC00020736563746F723A20256C64206174207E
:109ED000256C582025640D0A000D0A5772697465B7
:109EE00020256C642028256C582920733A256C6441
:109EF00020000D0A5365656B696E6720746F20251D
:109F00006C642028256C5829000D0A535338303AC8
:109F100020496E6372656D656E743A000D0A535385
:109F20003830783A436C656172000D0A414D3A440D
:109F3000534A000D0A535338303A4275666620770B
:109F40007220256C64206279746573207278000D2C
:109F50000A57726974655F736563746F7273206604
:109F600061696C202564000D0A47504942207263E4
:109F70003A25642025642062797465730D0A000D0A
:109F80000A53533830783A577269746520256C64E7
:109F90002028256C582920000D0A20256C64206299
:109FA000797465732073656E7420000D0A323A521D
:109FB0006561642072746E2025582C2025642072FF
:109FC00065616420000D0A566563746F7220256C0C
:109FD000642028256C582920000D0A313A52656109
:109FE000642072746E2025582C20256420726561CF
:109FF0006420000D0A53533830783A52656164206A
:10A00000256C642028256C582920000D0A536565AD
:10A010006B20746F20256C64206661696C65642018
:10A020002564000D0A52656164206265796F6E6473
:10A0300020656E64000D0A5365656B206265796F5B
:10A040006E6420656E64000D0A5365656B696E670A
:10A0500020746F20256C642028256C582920000D61
:10A060000A53533830783A5365656B3A20000D0A2D
:10A0700053533830783A53746174757320000D0A65
:10A0800053533830783A44657363726962652000CF
:10A090000D0A535338303A496E6974206469736B02
:10A0A000000D0A535338303A4E4F50000D0A5353A7
:10A0B00038303A536574206C656E67746820256C7F
:10A0C0005820000D0A535338303A536574206164A8
:10A0D000647265737320256C5820000D0A53533841
:10A0E000303A556E6B6E6F776E20255820000D0A42
:10A0F000535338303A527120737461747573200071
:10A100000D0A535338303A446573637269626500CF
:10A110000D0A535338303A53657420766F6C756D61
:10A1200065202564000D0A535338303A5365742076
:10A13000756E6974202564000D0A535338303A5700
:10A1400072697465000D0A535338303A5265616480
:10A15000000D0A535338303A436820696E64204337
:10A160006C65617220256420000D0A535338303A23
:10A17000416D69676F20436C656172202564200022
:10A180000D0A535338303A5270742051535441548D
:10A1900020256420002050503020005B4D4C415D54
:10A1A000005B4D54415D002050503120000D0A4DA0
:10A1B000617820566563746F7220256C64202825B1
:05A1C0006C582920008D
:0AA1C60081868A908A928A94938021
:10A1D000938293849568938C938E9388938A9386C5
:10A1E00092900001AD6BAE6B1F6A206AFF0E1F5C80
:10A1F000000E20580BE2000E1F24E96E010E2020F5
:10A20000EA6EEF6A1F2A000E2022F0D71F6A206A2A
:10A21000FF0E1F5C000E20580BE2000E1F24E96E9B
:10A22000020E2020EA6EEF6A1F2A000E2022F0D7CD
:10A230002F6A1200D9CFE6FFDACFE6FFE1CFD9FFD0
:10A24000E2CFDAFF2C6A216A226A080E8A148A6E2B
:10A2500093868A908A928A948A9893809382938430
:10A2600093889568FC0EDBCFE6FFFD0EDBCFE6FFA3
:10A27000760E006E9C0E016E026A00C0E6FFE66E6E
:10A2800002C0E6FF800EE66E000EE66E3BEC56F076
:10A29000036E070EE15C02E2E16AE552E16E0350F3
:10A2A000800EE66E000EE66E87EC54F0E552E55245
:10A2B000FC0EDBCFE6FFFD0EDBCFE6FF000EE66E09
:10A2C000020EE66E61EC3DF0E552E552E552E552D4
:10A2D000630E2C5C01E1D4D08150400B01E1D0D061
:10A2E0008150100B27E18150200B24E18050010B9D
:10A2F000E66EE66A6F0E006E9C0E016E026A00C08A
:10A30000E6FFE66E02C0E6FF800EE66E000EE66E29
:10A310003BEC56F0036E070EE15C02E2E16AE552A7
:10A32000E16E0350800EE66E000EE66E87EC54F090
:10A33000E552E552A00E236E860E246E010E256EA8
:10A34000266A2C50620A01E174D0640A62E0030AB2
:10A3500057E0010A4FE0070A45E0020A22E0030A3B
:10A3600020E0020AB5E18150020B61E08150040B4C
:10A370005EE023C000F024C001F025C002F026C03A
:10A3800003F02306000E245A255A265AD88000547A
:10A39000000E0154000E0254000E035499E3620EA5
:10A3A0006DD0FC0EDBCF00F0FD0EDBCF01F0000620
:10A3B000000E015A0050211807E10150221804E153
:10A3C000020E1E1401E0939A000E2124E96E020E83
:10A3D0002220EA6EEF1C8C6E212A000E2222956A42
:10A3E000030E0AD081A202D0040E2C6EF2A470D704
:10A3F000040E0DD09390050E2C6ED66AF29468D799
:10A4000081A402D0060E2C6EF2A462D7060E2B6E2B
:10A410005FD79568938A9380FC0EDBCF00F0FD0E2A
:10A42000DBCF01F00050215C0150225826E2010EE2
:10A4300025D0660EE66E9C0EE66E6C0E006E9C0ECF
:10A44000016E026A00C0E6FFE66E02C0E6FF800E03
:10A45000E66E000EE66E3BEC56F0036E070EE15C16
:10A4600002E2E16AE552E16E0350800EE66E000EF4
:10A47000E66E87EC54F0E552E552630E2C6E28D759
:10A480009380938293849388938A9568F70E9310B0
:10A49000936EE552E5CFDAFFE7CFD9FF1200D9CFAF
:10A4A000E6FFDACFE6FFE1CFD9FFE2CFDAFFE652EF
:10A4B000E652DF6AD00E276E070E286E296A2A6AD6
:10A4C0000001AD6BAE6B010EDB6A8A6A93868A90DF
:10A4D0008A928A94819281949380939293949568BE
:10A4E0002B6AE66AE66EE66A000EE66E010EE66E1E
:10A4F000F8EC54F0006E050EE15C02E2E16AE55210
:10A50000E16E0050630E2B5C01E1C5D00001000E2E
:10A51000AD5D010EAE5903E28150400B02E1090E20
:10A520002B6E2B50090A01E1B1D0030A01E1AAD038
:10A530000C0A01E192D0030A45E0010A3FE0070A54
:10A5400016E0010A0CE0030A05E0010ADBE1939240
:10A55000939481D09382D66AF294020E9AD081B0FD
:10A5600002D0030E2B6EF2A4CDD70A0E92D0D00EDD
:10A57000276E070E286E296A2A6A9392831CE66E5C
:10A58000000EAD25E96E010EAE21EA6EE552E750F0
:10A59000EF6E8150200B01E0010E2D6E8150100BEB
:10A5A00001E0010E2E6EAD2B000EAE230A0E236EBF
:10A5B000246A256A266A9384040E6BD081A0A2D7F0
:10A5C000050E67D093940F011F5118E02F50E66ECF
:10A5D0002E5002E0000E01D0010EE66EADC0E9FF84
:10A5E000AEC0EAFFE906000EEA5A000EE926010EA7
:10A5F000EA22EF50E66EE8EC19F017D02F50E66E25
:10A600002E5002E0000E01D0010EE66EADC0E9FF53
:10A61000AEC0EAFFE906000EEA5A000EE926010E76
:10A62000EA22EF50E66EDCEC2CF0E552E552E55202
:10A63000010EF3CFDBFFDB5027E12D500CE1060EBE
:10A640002B6EE80E236E030E246E256A266ADE52F8
:10A65000FE0EDD6E57D7010E1CD0938481AA02D066
:10A66000090E2B6E2306000E245A255A265AD8802E
:10A670002354000E2454000E2554000E265401E2EB
:10A6800041D702D0010EDF6E090E03D0939293944E
:10A69000630E2B6E37D72E5030E1ADC0E9FFAEC050
:10A6A000EAFFE906000EEA5A000EE926010EEA2248
:10A6B000EF50600822E1ADC0E9FFAEC0EAFF020E34
:10A6C000E95E000EEA5A000EE926010EEA22EF507A
:10A6D0005F0813E1020E1E101E6EAFC000F2B0C084
:10A6E00001F2020EE66EE66AA5DDE552E552FD0EC8
:10A6F0001E141E6E0001AD6BAE6B0001000ED88003
:10A70000AD55000EAE55DF5003E0F368F46A07D094
:10A71000010EDB50006E016AF36E01C0F4FFE552DA
:10A72000E552E552E5CFDAFFE7CFD9FF1200819C71
:10A73000939CA00E236E860E246E010E256E266A53
:10A74000235024102510261006E02306000E245A5C
:10A75000255A265AF5D7818C938CA00E236E860E2F
:10A76000246E010E256E266A235024102510261013
:10A7700006E02306000E245A255A265AF5D7120061
:10A78000D9CFE6FFDACFE6FFE1CFD9FFE2CFDAFF9C
:10A79000FD0EDB0403E19396819602D093868186B9
:10A7A000E552E5CFDAFFE7CFD9FF1200D9CFE6FFB8
:10A7B000DACFE6FFE1CFD9FFE2CFDAFFE652E65289
:10A7C000D650026E036AD750046E056A3F6A010EC6
:10A7D000406E04C044F005C045F05AEC57F00250FA
:10A7E0003D24006E03503E2000C0DEFFDD6EF250BF
:10A7F000040B01E0010EE66EE66ADECFE6FFDDCF78
:10A80000E6FFFD0EDBCF00F0016A00BE016800C06C
:10A81000E6FF01C0E6FF5B0E026E9C0E036E046A4B
:10A8200002C0E6FFE66E04C0E6FF800EE66E000E94
:10A83000E66E3BEC56F0056E0B0EE15C02E2E16A5F
:10A84000E552E16E0550800EE66E000EE66E87EC76
:10A8500054F0E552E552F294E552E552E552E5CF67
:08A86000DAFFE7CFD9FF120077
:08A868000C0EAF6EB06AB89649
:10A87000AC98AB8EAB88AB9A9D989D9AD08E9F8AF0
:10A88000F28EAC90AB9CAC9AAC8AAC9404018191F2
:10A89000806B1200D9CFE6FFDACFE6FFE1CFD9FF18
:10A8A000E2CFDAFFACA2FED7FD0EDBCFE6FFABECCA
:10A8B00057F0E552E552E5CFDAFFE7CFD9FF1200B6
:10A8C0009EBA03D0040007D8FBD7AE5000D01200C8
:10A8D0009EBA010C000CD9CFE6FFDACFE6FFE1CF3C
:10A8E000D9FFE2CFDAFFE652ABA204D0AC9AAC8A31
:10A8F000AB98AB88ABA404D0AE50DF6EAC9AAC8AF8
:10A90000E552E552E5CFDAFFE7CFD9FF1200D9CF04
:10A91000E6FFDACFE6FFE1CFD9FFE2CFDAFF0401AD
:10A92000826B836BFC0EDBCFE9FFFD0EDBCFEAFF12
:10A93000EF5014E0FC0EDBCFE9FFFD0EDBCFEAFFAA
:10A94000EF50E66EA7DFE552FC0EDB2AFD0E01E3B9
:10A95000DB2A0401822B000E8323E4D7280E83AF69
:10A9600002D0D89003D0825D000E835910E3230EED
:10A97000E66E90DFE5524F0EE66E8CDFE552460E36
:10A98000E66E88DFE552230EE66E84DFE552E5527F
:0AA99000E5CFDAFFE7CFD9FF120090
:06A99A00D9CFE6FFDACF81
:10A9A000E6FFFA0EE3CFD9FFFB0EE3CFDAFFFC0E92
:10A9B000E3CFE9FFFD0EE3CFEAFFE9CFF3FFEACFF4
:10A9C000F4FFF80EE35003E1F90EE35008E0F80E4F
:10A9D000E30602E2F90EE306DECFEEFFF2D7FF0E4A
:10A9E000E3CFDAFFE552FF0EE3CFD9FFE5521200C5
:10A9F000FE0EE3CFE9FFFF0EE3CFEAFFE9CFF3FF5F
:10AA0000EACFF4FFFB0EE35003E1FC0EE35009E054
:10AA1000FB0EE30602E2FC0EE306FD0EE350EE6ED3
:10AA2000F1D71200FD0EE3CFF6FFFE0EE3CFF7FFE6
:10AA3000FF0EE3CFF8FFFB0EE3CFE9FFFC0EE3CF01
:10AA4000EAFFEE500900F55C02E1F566FAD7120064
:10AA5000FE0EE3CFE9FFFF0EE3CFEAFFF36AF46AED
:10AA6000EE5203E0F34AF42AFBD71200FF0EE3CFC5
:10AA7000F8FFE552FF0EE3CFF7FFE552FF0EE3CFFD
:10AA8000F6FFE552E66AE66AE66A0900F55209E071
:10AA9000FD0EE32A05E1FE0EE32A02E1FF0EE32AA2
:10AAA000F4D7FD0EE3CF3EF0FE0EE3CF3FF0FF0EF6
:06AAB000E3CF40F01200AC
:0AAAB600FF0EE3CFEAFFE552FF0EAA
:10AAC000E3CFE9FFE552E66AE66AD9CFE6FFDACFDF
:10AAD000E6FFFC0EE124D96EFF0EE220DA6EE66A94
:10AAE000E66AE66A200EEF5C06E0090EEF5C03E022
:10AAF000EF6603D03FD0EE50F5D72D0EEF5C03E1AB
:10AB0000FF0EE32A03D02B0EEF5C01E1EE502F0E77
:10AB1000EF6424D03A0EEF6021D0D890F90EE336DE
:10AB2000FA0EE336FD0EDECFE3FFFE0EDDCFE3FFD0
:10AB3000D890F90EE336FA0EE336D890F90EE336E4
:10AB4000FA0EE336FD0EE350DE26FE0EE350DD2264
:10AB5000300EEE5CDE26000EDD22D9D7FF0EE3CFED
:10AB6000E8FFE85207E0F90EE31EE32AFA0ED8B434
:10AB7000E306E31EE552E552E552FF0EE3CFDAFFAE
:10AB8000E552FF0EE3CFD9FFE552E1CFE9FFE2CF77
:10AB9000EAFFED52ED52EECFF3FFEFCFF4FF1200DC
:10ABA000D9CFE6FFDACFE6FFE1CFD9FFE2CFDAFF78
:10ABB000E652E652DE6ADD6ADECF00F0DDCF01F05C
:10ABC000FC0EDBCF02F0FD0EDBCF03F00250005C89
:10ABD000035001580AE2080EE66ED4EC57F0E55235
:10ABE000DF2A010EE9E3DB2AE7D7E552E552E55219
:10ABF000E5CFDAFFE7CFD9FF1200D9CFE6FFDACFF2
:10AC0000E6FFE1CFD9FFE2CFDAFFE652E652DE6A95
:10AC1000DD6ADECF00F0DDCF01F0FC0EDBCF02F00D
:10AC2000FD0EDBCF03F00250005C035001580DE233
:10AC30000000000000000000000000000000000014
:10AC4000DF2A010E01E3DB2AE4D7E552E552E552A3
:10AC5000E5CFDAFFE7CFD9FF1200C2900F0EC16E29
:10AC6000070EB46ED36A4F0EC86E946A94889482AD
:06AC70009484826A1200C8
:0AAC7600D9CFE6FFDACFE6FFE1CF09
:10AC8000D9FFE2CFDAFFE652E652E652E652D95059
:10AC9000F90F006EFF0EDA20016E020E00C0DBFF1E
:10ACA000030E01C0DBFF020EDBCFE6FF030EDBCF9E
:10ACB000E6FFF90EDBCFE6FFFA0EDBCFE6FFFB0E79
:10ACC000DBCFE6FFD950FC0FE66EFF0EDA20E66E12
:10ACD0002FEC43F0006E070EE15C02E2E16AE55200
:10ACE000E16E0050F3CFDEFFF4CFDDFFFC0EDBCFD3
:10ACF000E9FFFD0EDBCFEAFFEF6ADECF00F0DDCF2C
:10AD000001F000C0F3FF01C0F4FF040EE15C02E2B9
:10AD1000E16AE552E16EE552E5CFDAFFE7CFD9FF10
:02AD200012001F
:0EAD2200060EF66E000EF76E000EF86E0F01B4
:10AD30000900F5501A6F0900F5501B6F03E11A67FF
:10AD400001D03DD00900F550156F0900F550166F80
:10AD50000900F550176F09000900F550E96E090068
:10AD6000F550EA6E090009000900F550186F090056
:10AD7000F550196F09000900F6CF1CFFF7CF1DFF32
:10AD8000F8CF1EFF15CFF6FF16CFF7FF17CFF8FF4E
:10AD90000F01185302E1195307E00900F550EE6E58
:10ADA0001807F8E21907F9D71CCFF6FF1DCFF7FFF8
:10ADB0001ECFF8FF0F011A07000E1B5BBFD7120052
:10ADC000D9CFE6FFDACFE6FFE1CFD9FFE2CFDAFF56
:10ADD000FB0EDBCF00F0FC0EDBCF01F00001800E9C
:10ADE00001141AE1FB0EDBCFE9FFFC0EDBCFEAFF1B
:10ADF000EECFF3FFEDCFF4FFEE2A000EEF22F3CFFC
:10AE0000E9FFF4CFEAFFFD0EDBCFEFFFEF50016A61
:10AE1000F36E01C0F4FF10D0FB0EDB50FE0806E11C
:10AE2000FD0EDBCFE6FF02EC58F005D0FD0EDBCFC8
:10AE3000E6FF19EC58F0E552E552E5CFDAFFE7CF2F
:04AE4000D9FF120024
:0CAE44003D504202F3CF39F0F4CF3AF059
:10AE50004302F3503A26000EF4203B6E3D5044026C
:10AE6000F3503B26000EF4203C6E3D504502F3505B
:10AE70003C263E504202F3503A26F4503B22000E4C
:10AE80003C223E504302F3503B26F4503C223E50BD
:10AE90004402F3503C263F504202F3503B26F4500C
:10AEA0003C223F504302F3503C2640504202F350B4
:04AEB0003C2612002A
:0CAEB40040C04AF03FC049F03F5044024B
:10AEC000F4CF3EF0F3CF3DF040504502F4CF40F0D8
:10AED000F3CF3FF04402F3503E26F4503F22E86A9D
:10AEE000402249504502F3503E26F4503F22E86A82
:10AEF000402245AE80EF57F049503F5E4A50405ADD
:0EAF00004AAE000C44503F5E4550405A000CD3
:02AF0E003C6A9B
:10AF10003B6A3A6A396A200EE76ED8903D363E3673
:10AF20003F36403639363A363B363C364250395C4D
:10AF300043503A5844503B5845503C5809E342501E
:10AF4000395E43503A5A44503B5A45503C5A3D2A88
:06AF5000E72EE4D7120019
:0AAF5600D9CFE6FFDACFE6FFE1CF26
:10AF6000D9FFE2CFDAFFACAC04D0AC900001FFB364
:10AF7000AC80FD0EDB50AD6EE552E5CFDAFFE7CFDA
:04AF8000D9FF1200E3
:0CAF8400F36AF46AFF0EE124E96EFF0E90
:10AF9000E220EA6EED6607D02F0EEF6404D03A0E81
:08AFA000EF6001D0F32A12005A
:08AFA800FF0EE3504B6E480E52
:10AFB00001D04C0EE76EE72EFED7E76AE72EFED7EC
:08AFC0004B2EF7D70000120030
:08AFC800800EF36E00EE00F0B4
:10AFD0000F0E01D81200EA6002D0EE6AFCD7F350DF
:08AFE000E9601200EE6AFCD7E3
:08AFE8001EEE00F02EEE00F059
:10AFF000F86A389C91EC56F01AEC58F0A8EC39F04D
:04B00000FBD7120068
:0CB00400FF0EE350ACBA04D0AF6AAB8E74
:10B01000AC8A949CACA2FED7AD6EF36EF46A1200BB
:10B0200030313233343536373839616263646566BE
:01B03000001F
:01B03100FF1F
:02B0320012000A
:02B03400120008
:0AB036002F6C6966646174612E627C
:10B04000696E20002F68706469736B2E63666700F9
:01B0500000FF
:0FB05100800102E805000913400100010001F62B
:10B06000008C119411941F010000000000000000EA
:10B07000000000E34007000000003F005F012001E6
:0EB080006501200040003400370000000A0087
:02B08E00800040
:10B090004C4142454C31000000028000000000009D
:10B0A000000E00004D5946494C4531323334000101
:10B0B0000000000100002000131012000000010039
:08B0C000000000000000000088
:020000040030CA
:0100010006F8
:0100020019E4
:010003001EDE
:010005008179
:010006008178
:00000001FF
